:020000020000FC
:0200000037C007
:02000800567828
:100034000C94EC290C94EA294156522D43686970BA
:100044004261736963322028632920323030362DAF
:1000540032303038204A6F65726720576F6C667291
:04006400616D0000CA
:10007000F894A0E02A2EA1E03A2EA0E1AEBFAFEFA7
:10008000ADBFB0E0A0E0AA95F1F7BA95D9F70E940C
:100090007C2B0E947A370E940E790E944B330E947B
:1000A000D62CAFEFA093310120923D0120923E016A
:1000B000209250018827789420922D01A091290147
:1000C000A4FD0C946A000E94D62C0E9490010E940C
:1000D0003231CECFA1E00E944C2CAA270E94F62BF1
:1000E0009927A7E10E94472C0E94D62CA0E10E94EC
:1000F000472CC4E0DAE0E7E3F7E10E941A30A7E01A
:100100000E94472C0E94CB2E0704200070D1A6E14C
:100110000E94472CC5E0D8E0E6E0F9E00E941A30E2
:10012000D8E1F9E10E941A30D8E0F9E0CC5FEC5F49
:10013000C833A0F366E90E9409316A95E1F70C948F
:10014000A100A0E00E944C2CA1E00E94BE329927A1
:1001500020922A01AA270E94F62BA5E10E94472C93
:100160000E94D62CC0E0D0E0EDE1F4E10E946E30B8
:10017000A1E50E94472C0E94CB2E0101838383833B
:100180008383204156522D436869704261736963CD
:1001900032208282828282820000A9E9B4E00AE4ED
:1001A0000D9304EC0D930CE80D9308E20D9302E619
:1001B0000D9306EA0D93509606EA0D9302E60D9311
:1001C00008E20D930CE80D9304EC0D930AE40D93F3
:1001D000F4D140913D014B3008F0442740933D015C
:1001E000642F67FD66276B3008F06AE050E06F937C
:1001F00011D16F9153955830D1F7B5D18AD15FD1D4
:100200006F935ED26F91423E11F46A95EACF433EFE
:1002100011F46395E6CF443E21F4643010F064504D
:10022000E0CF453E21F4673010F46C5FDACF6830E0
:10023000F8F04A3E11F0443F19F760933D016830F1
:1002400039F44A3EE9F6E1D00E94771BDED079CF3F
:10025000693039F44A3EA1F6D8D00E941420D5D096
:1002600070CFD3D04A3E61F60E94A721CED069CF8D
:100270004F934091140142FD2AC04F914A3E11F024
:10028000443F41F460933D01C0D088270E94900113
:10029000BCD057CF413F41F460933D01B6D0882791
:1002A0000E947A01B2D04DCF423F39F460933D01B4
:1002B000ACD00E94251DA9D044CF433F39F46093B0
:1002C0003D01A3D00E948A1DA0D03BCF99CF4F9172
:1002D000423F39F460933D0198D00E94760395D057
:1002E00030CF443F99F760933D018FD00E94BE0309
:1002F0008CD027CFA0911601A030E1F70E943204E4
:1003000020922D01A0911701A43F09F01ACF08D027
:100310000E943931A0E00E94F62B0E94D62CEACF31
:100320000E94D62C8827209216010E94D00D209280
:100330000D012092500120922A010E94102DA7E267
:100340000E94472C92E0A0913E01A03079F0A330AA
:1003500021F4A7E20E94472C09C0A0E10E94472C8B
:10036000A0E4A0930001A0EEA0930101A0913E01A2
:10037000A03051F40E94CB2E16002050524553530A
:100380002045534320002EC0A13051F40E94CB2EB3
:10039000690020505245535320455343200022C04A
:1003A000A23051F40E94CB2E4200205052455353AC
:1003B00020455343200016C0A33049F40E94CB2EA1
:1003C0002F00205052455353204553432000A53061
:1003D00049F40E94CB2E38002050524553532045FB
:1003E00053432000A0911601AD3EE1F708950E940D
:1003F000CB2EFF4156522D43686970426173696389
:10040000322056302E3835000895A0911601A030C4
:10041000E1F70895A1E0B3E050FDA95F51FDA25FAF
:1004200052FDBA5F4EE2651709F4429540932C01E4
:100430000E94E42E0E94CB2EFF20200040E50E9467
:100440003D2D452F4F5C0E943D2D0E94CB2EFF205D
:100450002000B3950E94E42E0E94CB2EFF2020D0D6
:10046000D1202000B3950E94E42E0E94CB2EFF20C5
:1004700020D2D3202000E0E0F0E950FDF45F51FDF0
:10048000F85E52FDF05DB3950E94E42E66E0459162
:100490000E943D2D6A95D9F7B3950E94E42E66E03F
:1004A00045910E943D2D6A95D9F7B3950E94E42E9F
:1004B0000E94CB2EFF2020202020200008954AE219
:1004C0006A3009F4429540932C010E94CB2E0F0F05
:1004D00020202020202000000E94CB2E100F202062
:1004E000D4D5202000000E94CB2E110F2020D6D77B
:1004F000202000000E94CB2E120F20494E464F2094
:1005000000000E94CB2E130F20202020202000006E
:10051000089548E2693009F4429540932C010E9405
:10052000CB2E0F0820202020202000000E94CB2E60
:1005300010082020D8D9202000000E94CB2E1108BE
:100540002020DADB202000000E94CB2E1208434F2F
:100550004E46494700000E94CB2E13082020202041
:100560002020000008954CE2683009F44295409341
:100570002C010E94CB2E0F012020202020200000E3
:100580000E94CB2E10012020DCDD202000000E94E4
:10059000CB2E11012020DEDF202000000E94CB2E78
:1005A000120144464C41534800000E94CB2E1301D7
:1005B00020202020202000000895A0E00E94472C49
:1005C0000E94CB2E1500202020202020202020203B
:1005D000202020202020202020202020202020201B
:1005E000202020200000A7E20E94472C0E94CB2E52
:1005F00016002020202020200000A0E60E94472C8A
:100600000E94CB2E16062045646974200000A0E4E9
:100610000E94472C0E94CB2E160C20536176652039
:100620000000A7E10E94472C0E94CB2E1612204CFE
:100630006F6164200000AEE6A0932B07A7E30E9441
:10064000472C0E94CB2E16182052756E200008955C
:10065000A0E00E94472CA7E20E94472C0E94CB2ECC
:1006600016002020202020200000A0E60E94472C19
:100670000E94CB2E16062020202020200000A0E47F
:100680000E94472C0E94CB2E160C20436F707920BD
:100690000000A7E10E94472C0E94CB2E16122020BA
:1006A000202020200000AEE6A0932B07A7E30E94A5
:1006B000472C0E94CB2E1618436C6561720008957A
:1006C0003DED209217010E94D631409114014470F3
:1006D000431739F0342F403011F46FDFF4CFB8DF17
:1006E000F2CF40911701403071F30895A4E00E94C9
:1006F000472CC1E0DFE0ECE1F3E10E946E30A0E4C2
:100700000E94472C0E94CB2E1002436F707920501C
:10071000726F6772616D20746F0070913D0160E0CF
:10072000ACE0671709F4A0E60E94472CB2E1A62FBF
:10073000AA0FA60FAD5F0E94E42E40E50E943D2D5A
:10074000462F47704F5C0E943D2D6395683041F7FE
:100750000E943231423E21F47030D1F37A95DFCFDE
:10076000433E21F47730A1F37395D9CF4A3E19F473
:100770000E94357A08954D3E59F708950E94A83594
:100780004F436C65617220746869732050726F67A3
:1007900072616D3F2000413009F008950E94167A81
:1007A0000895AA270E944C2CA3E00E94BE328F938A
:1007B00040913D010E9415790E94D62C0E94EB2B9E
:1007C0009927409116014030E1F70E94CB2E00009E
:1007D0002050524F4752414D200040913D014F5C07
:1007E0000E943D2D4AE30E943D2DC3EDD1E059D238
:1007F000F1D20E94DA7904D48F91A8E8803069F1AF
:10080000ACECEAE3F0E1813031F0ABE48A9545915C
:100810004030E9F7F8CF4DD292E0A5E0B1E00E9478
:10082000E42E0E94C32E0E94CB2EFF20494E205062
:10083000000040913A014F5C0E943D2D4AE30E9426
:100840003D2DBB27AC2DA3950E94662C4AE30E9448
:100850003D2DAD2DA3950E94662C0895AAE25A2E37
:1008600070E208959927FADF9CDFD22CAA27BB27D4
:10087000D0922E010E945C310E94D631403E11F48C
:10088000AA27F6CF413E11F4AFE12BC0423E11F44E
:10089000AA9527C0433E69F4A3959B2F0E94560951
:1008A0009A1730F4BE3511F4AA951BC0AA27B39548
:1008B00018C0443E21F4BA95B7FDBB2712C0463E8E
:1008C00021F4B850B7FDBB270CC0473E11F4B85F08
:1008D00008C0453E11F4B39504C04A3E39F5B395BE
:1008E000AA27A03838F0AFE1BA95B038C0F0AA27EF
:1008F000BB27BECFA03228F0BE3589F0AA27B3951A
:10090000B7CFBF3508F0BEE50B2F0D1508F4D02E7C
:100910000D2D015F0B1718F40B2F0F50D02E9B2FAE
:100920000E9456099A1708F4A92FA2CF9B2F4E3E7A
:1009300039F4AF93BF930E941809BF91AF918AC158
:100940004F3E39F4AF93BF930E942309BF91AF91FB
:1009500081C1493E11F482D17DC14C3E31F4A030B9
:1009600009F488CFAA957AD175C1509114015470B9
:1009700009F4C5C0433FD1F4ACEC9BD10E94CB2E0F
:100980000107524543454956452050524F47524171
:100990004D20592F4E203F006DD12EF48DD230D3F3
:1009A0005DDF5092C8017DD1882760CF423F39F585
:1009B000ACEC7FD10E94CB2E010753454E44205012
:1009C000524F4752414D20592F4E203F000052D1E7
:1009D00056F7ACEC6ED10E94CB2E010753454E4426
:1009E000494E472E2E2E202020202020202000009F
:1009F00030922A0193D120922A0130DFD4CF443F94
:100A0000B1F4ACEC56D10E94CB2E0107434C4541CA
:100A1000522050524F4752414D20592F4E203F00F7
:100A200029D126F4DBD21ADF5092C801BCCF413F56
:100A300041F5ACEC3ED10E94CB2E01075052494EFD
:100A4000542050524F4752414D20592F4E203F00C5
:100A500011D1B6F4ABE42DD10E94CB2E0107505238
:100A6000494E54494E472E2E2E2020202020202053
:100A70002000A2E0A0932A0151D120922A01EEDEAB
:100A800092CF433671F462E46093E50165E56093CB
:100A9000E60166E46093E7016DE36093E80179D2D3
:100AA000E9CE483791F462E46093E50165E560932F
:100AB000E60166E46093E7016DE36093E8010E945C
:100AC000C9077CD25092C80118C04637B1F4609172
:100AD000E501623499F460E26093E5016093E60118
:100AE0006093E7016093E8016093E9016093EA0194
:100AF00043D286D25092C801BDCE8827BBCE423F9A
:100B000011F5BF93AF93C9D0D9F0ACECD2D00E940D
:100B1000CB2E0107534156452050524F4752414D6D
:100B200020592F4E203F0000A5D046F40E94A879FE
:100B30000E94DA7965D292DE7093C801B2D088271C
:100B4000AF91BF9195CE433FE1F4BF93AF93A5D052
:100B5000B9F0ACECAED00E94CB2E01074C4F5354F1
:100B6000204348414E47455320592F4E203F000017
:100B700081D026F70E94DA7943D270DE7093C801E3
:100B8000DDCF413F49F46A2E7B2EADD0A62DB72D87
:100B90005092C8016FCED2CF4D3E09F5BF93AF93AF
:100BA0007CD0A9F0ACEC85D00E94CB2E010751552A
:100BB000495420572F4F205341564520592F4E203E
:100BC0003F0058D046F7A0911601A030E1F70E94EF
:100BD000E32BA0E00E94F62BAF91BF910895443F14
:100BE000E1F45BD029F40E94E32B0E94D62C0895F7
:100BF000A9E65FD00E94CB2E010753415645204302
:100C000048414E474553204245464F524520525594
:100C10004E2100000E94323191CF5091140152FDBB
:100C20001CC053FD1AC04C31C0F04038B0F4AF3195
:100C300071F05A2FAFE10E94B1316A916983AA9590
:100C4000A517D9F74883A3955092C80113CE0E94E7
:100C5000B13148835092C8010DCE0CCE0E94B13103
:100C60005A2F5F3121F0498149935395FACF50E2D1
:100C7000588308950E943231493559F0493749F077
:100C80004A3E39F04E3439F04E3629F04D3E19F0D7
:100C9000F1CF68940895E8940895A091C801A03216
:100CA0000895A8E806D00E94CB2E01054F4B000006
:100CB0000895EF93FF939927A09340010E94CB2EB4
:100CC000010520202020202020202020202020205E
:100CD0002020202020202020202020202020200034
:100CE000FF91EF910895A0E00E9484314A3E09F4FB
:100CF0000895423E21F4A030B9F3AA95F5CF433EC2
:100D000021F4AB3089F3A395EFCF403268F340383C
:100D100058F74883AB3009F0A395E6CFC9ECD1E092
:100D200056E149910E943D2D5A95D9F70E94102D08
:100D30004EE511D016F04A95E1F7542F539544270C
:100D4000451719F024D04395FBCF43E20E943D2D77
:100D50000E94102D0895CF93DF935F936F93E894D3
:100D6000C4E3D2E053E2459FC00DD11D50E269912A
:100D7000613238F45A95D9F76F915F91DF91CF9135
:100D8000089568946F915F91DF91CF910895DF93FB
:100D9000CF934F935F936F93C1E3D2E053E2459FAC
:100DA000C00DD11DDF93CF93A39653E26A916132B8
:100DB00010F45A95D9F7CF91DF9149910E943D2DBA
:100DC0005A95D9F70E94102D6F915F914F91CF9155
:100DD000DF910895AF93BF93EF93FF934F93AEE0EE
:100DE000B2E0ECEFFDE04591403011F04D93FBCFC8
:100DF0004F91FF91EF91BF91AF9108952045786990
:100E0000742020204E616D6520202053617665207E
:100E10002052656C6F616420202052756E20200086
:100E2000AF93BF93EF93FF934F93AEE0B2E0E8E44C
:100E3000FEE04591403011F04D93FBCF4F91FF9173
:100E4000EF91BF91AF9108952020202020202020F5
:100E50005072696E74202053656E642020205265A4
:100E60006376202020204E6577202000AF93BF932B
:100E7000EF93FF934F93AEE0B2E0E4E9FEE04591DB
:100E8000403011F04D93FBCF4F91FF91EF91BF9107
:100E9000AF9108952041626F72742020202020209D
:100EA0002020202020202020202020202020202042
:100EB0002020202020202000D9DFACECFADE0E9488
:100EC000CB2E0105524543454956494E472E2E2EFD
:100ED000000020922E010E94EE079927ECECE0938F
:100EE0004001E3EDF1E0EE2EFF2E41E10E94C6321B
:100EF0005CE00E94E2324B31B9F14A33D1F70E94F3
:100F0000E2324B3189F1403218F041935A95B9F7EA
:100F1000403228F00E94E2324B3131F1F9CFEEE05D
:100F2000F2E0EE2EFF2E53E2EE2DFF2DB396EE2EC5
:100F3000FF2E0E94E2324B31B9F04032D0F34332FF
:100F400099F006C00E94E2324B3171F0403248F015
:100F500041935A95B9F70E94E2324B3129F0403261
:100F6000D0F793959036F9F60895A3E2BA9FA1E3DE
:100F7000B2E0A00DB11D0895BF93AF93F6DFC8E7AF
:100F8000D1E053E249914D935A95E1F7AF91BF916A
:100F90000895BF93AF93E9DFC8E7D1E053E24D91E5
:100FA00049935A95E1F7409178014093E9014091C6
:100FB00079014093EA01AF91BF910895BF93AF9338
:100FC0004F935F93D2DF139640E250E24D935A95D0
:100FD000E9F75F914F91AF91BF910895DF93CF9360
:100FE000BF93AF934F9340E2A1E3B2E0CDEFDCE0DB
:100FF0004D932197E9F74F91AF91BF91CF91DF9139
:10100000DF93CF93BF93AF934F9341E0A1E3B2E05F
:10101000C0E3D42FDA5010F0C395FCCFD65CCD934B
:10102000DD93C0E2CD9390964395403689F74F917A
:10103000AF91BF91CF91DF910895425245414B004E
:101040004F564552464C4F57004449564944452057
:101050002F30005351522046524F4D203C30004318
:101060004F4E5354414E5420544F4F204249470055
:1010700057524F4E472045585052455353494F4EB3
:101080000053594E544158204552524F5200554E2C
:101090004B4E4F574E204B4559574F5244005752D5
:1010A0004F4E4720464F524D415400424144204C40
:1010B000494E454E554D424552004E4558542057D5
:1010C0002F4F20464F520052455455524E20572F15
:1010D0004F20474F53554200544F4F204D414E59DA
:1010E00020474F53554200544F4F204D414E5920F9
:1010F000464F5200493243204552524F5200554EFE
:101100004B4E4F574E204552524F520044464C4191
:101110005348204552524F52004F5554204F4620BD
:10112000415252415900494E434F4D504C45544550
:1011300020504152004B4559574F524420495320AB
:101140004D495353494E470057524F4E4720424353
:101150004F505920004F5554204F4620534352457D
:10116000454E0043414E4E4F542043524541544555
:101170002046494C45004D454D4F52592046554C4F
:101180004C0046494C45204E4F5420464F554E4446
:101190000050414745204E4F5420494E2046494C6F
:1011A00045005041474553204E4F5420494E205250
:1011B000414E4745004E4F5420494E204752415022
:1011C00048494353204D4F4445004E4F5420494E0B
:1011D0002054455854204D4F4445004E4F20555300
:1011E000522046494C4500535243204F5554204FFE
:1011F000462053435245454E0044455354204F55D5
:1012000054204F462053435245454E0057524F4EAF
:10121000472053505249544500494F2044495341B7
:10122000424C4544004E4F204558544D454D00001A
:10123000BE3508F00895BF9328D0B395BE35E1F7C9
:10124000BDDEBF91DDCEBE3508F00895BF93AF93EC
:10125000AB2FAA95BDE508D0BA95BA17E1F7B395BB
:10126000ADDEAF91BF91CCCEBF93AF93DF93CF9361
:101270007CDE1396ED01B0E2A991AAA3BA95E1F73D
:10128000CF91DF91AF91BF910895BF93AF93DF935B
:10129000CF936BDE1396ED01B0E2ABA1A993BA95A3
:1012A000E1F7CF91DF91AF91BF910895BF93AF93D5
:1012B000DF93CF935ADEED0193964E914132E8F3DE
:1012C0004038D8F7AC1BBC0B9A2F925097FD99274A
:1012D000CF91DF91AF91BF910895CAEEDCE02A92E1
:1012E0002A9280E02F92AA27BB274427719170325F
:1012F000E9F37C3121F4A191BB27719156C07E3175
:1013000021F4A191BB27719150C07D3121F4B1919D
:10131000A19171914AC07F3121F4B191A191719154
:1013200044C07C3130F4572F4C2E5D2ECE2FDF2F52
:1013300063C07432C1F47191703320F07A3310F4C9
:10134000705305C0713468F0773458F47753B03176
:1013500048F4A295B2955A2F5F70A07FB52BA70FC6
:10136000EACF23C029C0703350F17A3340F54038BA
:1013700010F086E02AC1AA0FBB1FF0F04A2E5B2EA8
:10138000AA0FBB1FC8F0AA0FBB1FB0F0A40DB51D5C
:1013900098F07053A70FB21D78F0B7FD0DC0719192
:1013A000703318F07A3308F4E6CF4F3709F473D16D
:1013B000AA93BA9340E89DCF85E007C144C0713439
:1013C000E8F37B35D8F76081613458F16B3548F527
:1013D0004C2E5D2ECE2FDF2F21970C2F1D2FE4E4F6
:1013E000FBE152E07591703011F488E0EEC070328C
:1013F00061F46991683299F45F93452FAA27BB275E
:10140000EC2FFD2FC42DD52D71CF6991671751F3A6
:1014100075917032E9F75395C02FD12FE3CF87E054
:10142000D4C0403810F086E0D0C07154770FEF93ED
:10143000FF93E0E9FCE0E70FF21DA191B191FF916C
:10144000EF917191B2CF7D3251F44F3711F44427AF
:101450004DCF20F4403210F04FE748CF6FC07832C4
:1014600031F471E07F93AA27BB27472F3FCF793212
:1014700009F05EC05F91513019F0523011F403D180
:1014800053C0533011F413D14FC0543029F4CCD190
:10149000803009F09AC046C0553029F4B991A9911D
:1014A000B095A0953FC0563009F4DDC1573009F41E
:1014B0008DC2583009F49EC2593009F4B3C25A3073
:1014C00009F4C9C25B3009F4D1C25C3009F4D2C25C
:1014D0005D3009F4D4C25E3009F4AEC2503109F473
:1014E0000AC2513109F425C1523109F428C15331DE
:1014F00009F40EC2543109F423C25F3009F410C359
:10150000553109F4BCC1563109F4D0C1573109F441
:10151000D5C1503029F06ED0803009F056C0AACF26
:1015200086E00895AA93BA93AA27BB2742E0DECEAD
:101530004F3720F44F3010F086E047C07C3361F421
:1015400071E260816E3319F472E2619142C06D33D1
:1015500011F473E261913DC07E3339F474E260812D
:101560006D3311F475E2619134C07D3311F476E28C
:1015700030C07B3211F470E32CC07D3211F471E382
:1015800028C0733211F472E324C07A3211F470E48B
:1015900020C07F3211F471E41CC0753211F472E482
:1015A00018C0763211F473E414C05F91503021F00A
:1015B0005F3130F01FD0F9CFB991A99131970895DB
:1015C00086E05F915030C1F3FCCF4F914030E9F796
:1015D00008955F91A72FB52FA07FB07FBA1720F095
:1015E00009D0803091F7F5CF5F937F93AA27BB276F
:1015F000472F7CCE5F934F9319910991B991A9918F
:10160000513211F4FED03AC0523221F4F3D0A1503D
:10161000A17034C0533221F4FCD0A150A1702EC06F
:10162000543211F4F6D02AC0553221F4EAD0A15038
:10163000A17024C0563211F4DDD020C0503311F413
:1016400041D01CC0513311F43CD018C0523319F4AE
:10165000A02BB12B13C0503411F43FD00FC0513424
:1016600011F4A7D00BC0523421F4A3D0A22FB32F72
:1016700005C0533419F4A023B12300C0AA93BA9330
:101680004F915F910895B991A99103D0AA93BA930C
:101690000895B7FF0895A095B095A30DB21D0895C4
:1016A00017FF089500951095030D121D0895B99127
:1016B000A991AB2B29F0B7FBA1E0BB270EF4129741
:1016C000E5CFF0DF2B2F2127A00FB11F27FD0895B5
:1016D0002B2F212727FD82E008950CD0A22FB32FB6
:1016E000BF770EF4D8DF37FD03C0452B09F408950A
:1016F00082E008957AD0CDDFB19F402D512DA09F7B
:10170000202D312DA19F300D411D521DB09F300D58
:10171000411D521D089508E611E0B03818F0A00FE1
:10172000B11FFBCFA017B10718F0A01BB10BFACF68
:101730000895B991A9910AE5A01BB20902C0B99117
:10174000A991E9DFFF93EF93E2E2F7E70AE510E002
:10175000A017B10748F4E00FF11FEA1BFB0BA4919F
:10176000EF91FF91BB27DECE04EB10E0A017B1078D
:1017700078F40AE510E0E01BF10BEA0FFB1FA491DF
:10178000EF91FF91BB27A095B095A30DB21DCACED6
:101790000EE011E0A017B10728F4E00FF11FEA1BDB
:1017A000FB0BEDCF0EE011E0E01BF10BEA0FFB1F8E
:1017B000D6CF212F202B11F483E0089516D02227B5
:1017C0003327442751E1441FAA1FBB1F5A9551F0EC
:1017D000221F331F4FEF201B310BA8F7200F311FA3
:1017E00040E0F1CF0EF457CF08952B2F212727FB90
:1017F00050DF56CF0A271B27AA27BB27012B89F0CA
:101800000895B0581058A01BB10BAA27BB2748F069
:101810000895B05810580A1B1B0BAA27BB2708F0C5
:101820000895A1E0B0E00895B991A99184E0B7FDD1
:1018300008950F931F932F933F9388270A2F1B2FF1
:10184000B2E0AA27232D3327021B130B20F0A39508
:101850002B0F321DF9CFBB27AA93BA933F912F913B
:101860001F910F9108954F935F930E945A331991DE
:10187000099142DFA42FB52F5F914F9153CE19915B
:101880000991023039F420925001A2E0A093330173
:10189000BB2748CE013031F4A0913301A03011F4C0
:1018A00030923301A0913301BB273CCE19910991AD
:1018B0000EBD0E94CA17AEB5BB2734CE10913E01B3
:1018C000103011F08CE1089519910991A4ECB2E067
:1018D0000A171B0710F082E10895FF93EF93FDE0D4
:1018E000ECE3E00FF11F68940E94F932EF91FF9151
:1018F000A42FBB2717CEB991B0937301A991A093E0
:101900007201CF93DF930E94CE17DF91CF910ACE61
:10191000B991A991BF3F71F0A09358010E94F41FA3
:10192000803021F0AFEFBFEF8827FCCDA42FBB277D
:101930000C94920A0E94F91F8827B42FAA27F2CD8F
:10194000B991A991BF3F21F5A0FD11C0DF93CF93BD
:10195000FF93EF930E94F11F803019F08827CC2766
:10196000DD27DE01EF91FF91CF91DF91DBCDDF939A
:10197000CF93FF93EF930E94F11F803019F08827D7
:10198000EE27FF27DF01EF91FF91CF91DF91CACDC5
:10199000A09358010E94F41F803021F08827AA27C5
:1019A000BB27C0CDDF93CF937F9377270E94FC1F87
:1019B000DF3F41F4CF3F31F4A72FBB277F91CF9179
:1019C000DF91B0CD7395703889F7F6CFA991A991C1
:1019D000A770A06CA0937C00A0917A00A064A09353
:1019E0007A00A0917A00A6FDFCCFA0917800B0917A
:1019F000790098CDB991A991B03061F4AF3F79F0F9
:101A0000A770A395B0B1B695AA95E9F7AA27AA1F22
:101A1000BB2788CDBA2FA0B1AB23BB2783CDA0B104
:101A2000BB2780CDB991A99171E00E94C137803068
:101A3000C9F4BB27A52F76CDB991A991CF93DF9398
:101A4000CA2FDB2F0E94FE37DF91CF91803051F4F7
:101A5000BB27A42F67CDA99179910E94DC378030F4
:101A600009F460CDAA27BB278FE0ABCDB991A9912E
:101A7000BB2758CDB991A991AB2FBB2753CD0F935D
:101A8000B9910991AA27BB27003019F4A09116013A
:101A900045C0013029F4A0911601A030E1F33EC009
:101AA000023039F4A0911601A030E1F7A09117019E
:101AB00035C0033019F4A091140130C0043039F45A
:101AC0000091140100FD119602FD119727C0053009
:101AD00039F40091140101FD119603FD11971EC008
:101AE000063049F400911601023E09F41197033EB5
:101AF000A9F4119613C0073049F400911601043E71
:101B000009F41196053E51F4119708C01F931091E6
:101B100016010117E1F71F91A02FBB270F9102CDEE
:101B2000B991A991BB27A13021F4A0916D01A39592
:101B3000F9CCA23021F4A0916E01A395F3CCA09131
:101B40006F01F0CC4142532053474E205351522055
:101B50004E4F5420524E442041444320494E205879
:101B60005045454B2054454D50204C4F204849206E
:101B70004B455920455045454B2045525220415236
:101B80002053494E20434F53204654595045204638
:101B900053495A4520505354415420535049200032
:101BA000FCE0E0E9A0E0B4EBA193BA95E9F7F1E03D
:101BB000E8E6B0E1A193BA95E9F7FDE0ECE3B0E027
:101BC000A193A193A193BA95D9F7DD24CC242092B7
:101BD0000F0120920D01AEE0A0932C01ACE3A09385
:101BE0004401AEE2A0934501AFEFA09377010E94BC
:101BF000D62C20925001A2E0A0933301A6ECA09332
:101C00007A0040913D0140933A01409337010E9490
:101C100015799C2D0E9431791FD0803039F4AC2D7C
:101C2000AF35B8F39CE0209250010895C0926D0149
:101C3000D0926E0180936F01209250014091770104
:101C40004F3520F4DD24C42E8827E3CF9CE020927A
:101C500050010895F70129C0F1E0E0EA20922A013D
:101C60008827AD2DBB27AB1701F171917F3FC1F1E3
:101C70007C31C9F07E31B9F07D31A1F07F3191F036
:101C8000773271F1723241F471917F3F49F17732CD
:101C900039F17232C9F7E9CF7A3339F7B395AB1717
:101CA00021F703C071917191E0CF70912D0170FF08
:101CB00005C081E07E7F70932D01089572FF0BC0F7
:101CC000AB7F70932D01A0913E01A53011F0A030A3
:101CD00011F40E942E1B0E94D63171917F3F19F49E
:101CE000DD24C394089577FD2BC07032F1F27A336E
:101CF00011F4D394DACF773299F37134D8F07B357D
:101D000028F070527134B0F07B35A0F4672E0E9439
:101D100009177D3379F4E1DA803069F4762D715456
:101D2000770FDCE0C0E9C70FD21DA993B99393CF19
:101D3000EF91FF9187E00895703810F487E08ACF23
:101D40007F01E7EAFEE07F73E70FF21D099445C0CB
:101D5000EDC0A0C236C10CC1EDC22EC33BC736C315
:101D600037C33BC33EC38BC6A9C64CC3A2C3D4C2B0
:101D7000FAC32AC478C16CC47CC481C4E9C195C2C9
:101D800086C491C498C459C54AC1D5C077C22BC175
:101D9000E1C49BC426C3E2C403C54EC2DDC2C4C5B0
:101DA000A7C716C622C627C673C1A7C6F6C678C778
:101DB00028C637C65AC214C557C61FC181C297C3A9
:101DC00000C392C498C43DC175C13BC692C188E0AE
:101DD000089584E1089583E108950E940D179CE021
:101DE000732C20922A01B191B032E9F3BA3311F089
:101DF000BF3F59F4319770FC0E94102D40912A0189
:101E0000443010F00E94813726CFBB3311F4772481
:101E1000EACFBC3291F440912A01403031F40E9463
:101E20003C2DBA2DB770D9F706C00E943C2DB09159
:101E30002B01B770D1F77724D6CF732CB332C9F406
:101E4000209258012092590148DA4A2F40932A01E2
:101E5000443018F4433001F4C6CF0E94853768300F
:101E600051F550912A015E7F0E948737683119F53C
:101E7000BACFB03411F59DD740912A01433018F400
:101E80000E94E42EB0CF39F4A0935801B0935901C9
:101E9000A0932B01A8CF5FEF0E948737683259F4D7
:101EA0005A2F0E948737683231F45B2F0E948737A0
:101EB000683209F498CF8FE00895B13229F40DDA31
:101EC0009A2F91CF97CF8FCFB23241F441914F3FAC
:101ED000C9F34232C1F30E943D2DF8CFB63291F4DE
:101EE000FCD9B33010F082E10895CCE3DDE0CA0FF5
:101EF000DB1F4991403029F00E943D2D1196B330EF
:101F0000C0F371CFB53229F4E8D94A2F0E943D2D94
:101F10006ACF3197E2D9803009F00895903818F4EB
:101F20000E94662C60CF0E94C12C5DCFA0E0F3D64A
:101F30000E94D62C8FCEA2E0EED6A030C1F0A13008
:101F400059F0A0915A01A770AA0FB0912C01B77057
:101F5000A295BA2BB0932C01A0915801A770AA0F9B
:101F6000B0912C01B07FBA2BB0932C0173CE33CF3C
:101F7000A3E0D1D6A33018F1A0915801B091590136
:101F8000A0937201B0937301A0915A01B0915B01CB
:101F9000A0935801B0935901A0915C01B0915D01EB
:101FA000B03011F4A03051F00D010E94CE170E9404
:101FB0006217D001803021F41197F2CF4BCE0BCFB6
:101FC0000895A5E0A8D6A43068F0B3D77F93E0D6F3
:101FD000E0936B01F0936C010E94F82F7F91709356
:101FE0002C0138CEF8CEA1E096D6A130D8F340919E
:101FF0005801417040930D012DCEA5E08CD6A43040
:1020000068F097D77F93C4D6E0936B01F0936C018F
:102010000E941A307F9170932C011CCEDCCEA5E07B
:102020007AD6A43068F085D77F93B2D6C0936B017F
:10203000D0936C010E94F5347F9170932C010ACEED
:10204000CACEA5E068D6A43068F073D77F93A0D637
:10205000C0936B01D0936C010E9445357F917093C2
:102060002C01F8CDB8CEA3E056D6A23080F061D7CF
:102070007F93B0915801A0915A01A0936B01B09346
:102080006C010E94F72E7F9170932C01E3CDA3CEBB
:10209000A5E041D6A43068F04CD77F9379D6E09381
:1020A0006B01F0936C010E94D4307F9170932C01EE
:1020B000D1CD91CEA0913E01A03011F08CE10895D8
:1020C000A1E029D6A130A8F3A0915801B0915901FF
:1020D000CCE3DDE0CA0FDB1F40912C014F93AF92A0
:1020E000BF920E948C35BF90AF904F9140932C01CE
:1020F000B1CDA0913E01A03011F08CE1089572D6CF
:10210000C0937001D093710184D67C32F9F4A1E0C0
:1021100003D6A13070F2A0915801B0915901CCE3DF
:10212000DDE0CA0FDB1F40912C014F93AF92BF92AD
:102130000E94B535BF90AF90C0917001D0917101F0
:10214000499329924F9140932C0184CD87E082CD11
:10215000A0913E01A03011F08CE1089543D6C093C8
:102160007001D093710155D67C3281F7A1E0D4D5AE
:10217000A13009F030CEFF93EF93AF92BF92409120
:102180002C014F937F934F7040932C010E94931921
:10219000C1E0D2E0ECE1F5E10E946E30C0912C018B
:1021A000C295C0932C010E94CB2E03020000A09187
:1021B0005801B0915901CCE3DDE0CA0FDB1FA6E165
:1021C0004991403230F0403820F40E943D2DAA95CC
:1021D000B9F7772761E025D00E94B919623079F408
:1021E000C0917001D0917101799329927F914F91A3
:1021F00040932C01BF90AF90EF91FF912BCD7F9139
:102200004F9140932C01BF90AF90EF91FF91C091FF
:102210007001D09171014FEF499349931BCD87E035
:1022200019CD0E94AD178827603009F408950E94E7
:10223000C91D882762E00895A3E06DD5A230A0F003
:1022400078D67F93D0916C01C0916B01F0915801C9
:10225000E0915A01E0936B01F0936C010E94D4303D
:102260007F9170932C01F6CCB6CDA4E054D5A43068
:1022700021F48ED50E94D02FEDCCADCDA1E04BD571
:10228000A13090F0A0915801A295AA0FAF7EA09323
:102290000F01E0CCA1E03FD5A13030F0A091580172
:1022A000A150CA2EDD24089596CDA1E034D5A130E9
:1022B000D8F3A0915801A150A0937701CBCC8BCD3E
:1022C000A5E029D5A23030F1F1E0E0915801E770A6
:1022D000B0915A01B770BB0FB295B193A230C9F05B
:1022E000E770B0915C01B770BB0FB295B193A330AA
:1022F00081F0E770B0915E01B770BB0FB295B193FA
:10230000A43039F0E770B0916001B770BB0FB2959F
:10231000B193A0CC60CD5FCDA1E0FDD4A130D8F3C6
:10232000A0915801A53009F0A3700E94F62B0E94DD
:10233000D62C90CCA1E0EFD4A13068F0A091580148
:10234000B0915901B03019F4A03009F483CC0E9447
:1023500009311197F7CF3FCD20925001A2E0A09311
:102360003301A3E0D8D4A33020F1CCE3DDE0A09189
:102370005801B0915901B330E8F4AC0FBD1FA093E0
:102380005201A0935401B0935301B0935501A09111
:102390005A01B0915B01B33068F4AC0FBD1FA0933C
:1023A0005601B0935701A0915C01A0935001209277
:1023B000330150CC82E14ECC20925001BF91BF91AD
:1023C00008952DD5AB2B09F48BCC45CC26D543CC29
:1023D000F701EFD40E94E42E3ECC21D50E941231A9
:1023E0003ACC672F6F931BD56F914A2F0E943D2DDA
:1023F00065FD0E94BA310ED57C3271F70AD50E9474
:102400006D09F3CFA2E087D4A13019F0A23021F1F9
:10241000E2CCA0915801AA95AF3510F08AE01ACC11
:10242000B0916F01BF3010F08DE014CCAF93CCEEC3
:10243000DCE0A5E0AB9FC00DD11DB395B0936F015B
:10244000BD2DB395B068B993BC2DB993B0913D0142
:10245000B993DD24CF900895A0915A01AA95AF3584
:10246000E8F6B0915801BA95B770B0933701B091C2
:102470006F01BF3010F08DE0EDCBAF93CCEEDCE020
:10248000A5E0AB9FC00DD11DB395B0936F01BD2DDD
:10249000B395B068B993BC2DB993B0913A01B99393
:1024A000DD24CF904091370140933A010E94157985
:1024B0000895B3D4B0916F01B03011F48CE0089559
:1024C000BA95CCEEDCE0A5E0AB9FC00DD11DB0937A
:1024D0006F01B991B7FFF2CFBF77DB2EC990499159
:1024E00040933A010E941579089587E0089595D4A4
:1024F00090D47134D0F37B35C0F77154770F672EC9
:1025000088D47D3391F70E946D09803009F00895D9
:10251000DCE0C0E9C60DD21DA993B9937AD4743515
:1025200021F771917F3409F70E946D094A2E5B2EC5
:10253000803009F00895B0916F01BF3010F08EE047
:102540000895CCEEDCE0A5E0AB9FC00DD11DB395A6
:10255000B0936F01BD2DB395B993BC2DB99369921A
:102560004992599278CB59D4B0916F01B03011F49F
:102570008BE00895BA95CCEEDCE0A5E0AB9FC00DF2
:10258000D11DB991B7FDF4CFBF77B0936A015990CF
:102590007991BCE0A0E9A70FB21D0D911D91030D2B
:1025A000121D1E930E93A991B99111960A1741F429
:1025B0001B1731F4B0916F01BA95B0936F014BCBFB
:1025C000C52CD0906A010895A0913E01A03011F071
:1025D0008CE1089522D4BFEFB0937801B191B0326D
:1025E000E9F34B2FBF3F21F40E94102D319733CBDD
:1025F000BA33D1F3BB3391F3BC3231F40E943C2D9A
:10260000BA2DB770D9F7EACFB23241F441914F3FBA
:1026100059F3423219F30E943D2DF8CFB134B0F096
:10262000BB35A0F4B154BB0FB0936A01B081B13493
:1026300018F0BB3508F40AC0F5D3DCE0C0E910910E
:102640006A01C10FD21DA993B993C8CF87E008953D
:10265000E6D3803009F0FFCA4A2F4B2BE1F34091BB
:1026600022014030E1F3409122014030E1F711971F
:10267000F3CFD5D3A0932301B0932401EDCFB2D3F0
:10268000A0912301A993A0912401A993E4CAC7D3DF
:102690004A2F0E94C632BED37C3221F4BAD30E94A4
:1026A0006D09F6CFD8CA0E94D232A42FBB279AD385
:1026B000A993B993D0CAF70188D34A2FD73020F411
:1026C000C03D10F40E940738C6CAF7017ED35A2FC6
:1026D000AC2FBD2F71E00E94CF370E9409310E94BC
:1026E00009310E940931B7CA70910C0174FD30C0E4
:1026F00096D3A1B9B0CA70910C0174FD29C0F7013D
:1027000064D3D030B1F4BC2FB770B39577276FE79F
:10271000A0FD70E8A0FD6FEF77FB770F70F967FB06
:10272000660F60F9BA95C1F702B1072B062302B90B
:1027300092CAD13041F4B2B1C095BC23C095CA232E
:10274000BC2BB2B988CAD230E9F70E94BB1783CA42
:1027500082E2089564D30E94BE327DCA43D3C093FF
:102760007001D093710109911991105852D37C32A4
:10277000A9F42BD3B058D058C017D10710F00C2FA4
:102780001D2FA017B10710F40A2F1B2FD091710134
:10279000C09170011058099319935DCA86E008959D
:1027A000A0913E01A03011F08CE108951BD3C0939D
:1027B0007001D09371012DD37C3281F7FAD2C8EC2D
:1027C000D1E07EE17B9FC00DD11DCA0FD21DBB277A
:1027D000A881D0917101C0917001A993B9933BCAAE
:1027E000A0913E01A03011F08CE10895FBD2C0937E
:1027F0007001D09371010DD37C3281F6DAD2C8EC2E
:10280000D1E07EE17B9FC00DD11DCA0FD21DA2EB8E
:10281000CA0FA2E0DA0FBB27A881A695BA2FA77727
:10282000B295B078AB2BBB27D0917101C0917001EC
:10283000A993B99310CA86E00895D4D2C0937001C9
:10284000D0937101E6D27C32B1F7B3D2C8ECD1E0BB
:1028500070913E017370703021F5AF93BF93A695D0
:10286000B6957EE17B9FC00DD11DCA0FD21D788128
:10287000BF91AF91A0FD7695B0FD7695B0FD7695B0
:10288000A2EBB2E0CA0FDB1FAC9170FDA295A6953A
:10289000A770BB27D0917101C0917001A993B99322
:1028A000DAC97130D1F4AF93A695A695A69575E1D6
:1028B0007B9FC00DD11DCA0FD21D7881AF91A2FDA3
:1028C0007295A1FD7695A1FD7695A0FD7695717026
:1028D000D1E0C72FA881A295DACF7130F1F7AF937D
:1028E000A695A6957EE17B9FC00DD11DCA0FD21D76
:1028F0007881AF91A1FD7295A0FD7695A0FD7695AA
:102900007370D1E0C72FA881A295C1CFAF93A695D0
:102910007AE27B9FC00DD11DCA0FD21D7881AF9185
:10292000A0FD7295A72FB3CFA0913E01A03011F06A
:102930008CE10895A3E0EFD1A33080F0A09158017D
:10294000B0915901B33010F082E10895B23039F4FA
:10295000A73F28F082E1089581E208953CCACCE3C4
:10296000DDE0CA0FDB1FC0934601D0934901AC8163
:10297000A03091F3AE3180F7BB81B03069F3B7314D
:1029800058F7C0915801D09159012596BA9F000C73
:10299000111C000C111CC00DC11DD330E8F6D091E4
:1029A0005A01C0915C01C0934801D0934B01CF3FC5
:1029B00051F0DF3F41F0CA0FCA95CE3138F4DB0F3A
:1029C000DA95D73118F40E94273644C986E1089574
:1029D000A0913E01A03011F08CE108951ED2A0918B
:1029E0002D01A460A0932D0136C9A0912901A062F8
:1029F000A093290130C9A0912901AF7DA09329019D
:102A00002AC9A3E088D1A33009F0E5C90E94F41FC8
:102A1000443111F08EE108950E9408208030D9F7EA
:102A200019C9A3E078D1A33009F0D5C90E94F41FD9
:102A3000443111F08EE108950E940B208030D9F7C7
:102A400009C9A2E068D1A23009F0C5C9A4E1A093E8
:102A50005C010E940220803009F4FCC808950E94A5
:102A60000520803059F4F6C8A1E055D1A13009F015
:102A7000B2C90E94F41F443191F38EE10895A2E09F
:102A80004AD1A23009F0A7C9A0915801B0915901CB
:102A900040915A01CCE3DDE0403041F0D395413024
:102AA00029F0D395423011F082E108950E946F38E9
:102AB0000E945E39803009F00895CCC8A2E02BD185
:102AC000A23009F088C9A0915801B09159014091F4
:102AD0005A01CCE3DDE0403041F0D395413029F09C
:102AE000D395423011F082E108950E9428390E9466
:102AF0008B38803011F308954EC0F7013ED1A0937A
:102B000074010E9485376830B9F790FF28C0592FAB
:102B10000E948737603481F7A030C9F0DDE0CCE354
:102B2000409174014B0F4A1BC40FD21DA13039F0E4
:102B30000E948B37603579F55883AA95EFCF0E94B4
:102B40009037683541F558830E94813784C80E94C8
:102B50008B375030A1F350937401A52FDFCF592F3D
:102B60000E9487376831B9F43A2FDDE0CCE3409119
:102B700074014B0F4A1BC40FD21D5881503011F401
:102B8000303031F00E948737683229F4AA9569F70E
:102B90000E94813760C88FE0089541D1A093580109
:102BA000B093590137D17C3249F4319632D1723227
:102BB00031F031970E946D0985D1F4CF4CC87191E5
:102BC000723231F07F3F21F0BB27A72F7BD1F7CFA7
:102BD0007081E8CFA0913E01A03011F48DE10895FD
:102BE000A7E099D0B0915801B0934C01B13039F0C1
:102BF000B23009F1B33009F43CC085E10895A73043
:102C0000E1F7C8E5D1E0BA81B0934901BC81B09346
:102C10004601BE81B0934A01B885B0934701BA8599
:102C2000B0934B01BC85B09348010E947F33803044
:102C300009F008950FC8A63001F7C8E5D1E0BA81C0
:102C4000B0934901BC81B0934601BE81B0934A0163
:102C5000B885B0934701BA85B0934801BB85B0935E
:102C60004B010E947F33803009F008950C942A0EA6
:102C7000C4CFA430E9F7C8E5D1E0BA81B0934601EA
:102C8000BB81B0934901BC81B0934B01BE81B0932D
:102C900048010E947F33803009F008950C942A0E79
:102CA000A0913E01A03011F08CE10895F7018DD084
:102CB000C0935801D093590150917401A51708F49D
:102CC0005A2FA8E7B1E0503071F04D91A0937501F3
:102CD000B0937601A42FBB27F5D0A0917501B091D8
:102CE00076015A95F0CFAA27BB27ECD00C942B0E77
:102CF000A0913E01A03011F08CE10895A1E00BD02D
:102D0000A13040F0A09158014A2F43700E94F5363F
:102D10000C942A0E60C8F701A03009F40895DF93DF
:102D2000CF93C8E5D1E040E05A2F503029F4A42FCA
:102D30007F01CF91DF910895DF93CF934F935F93FE
:102D40000E946D095F914F91CF91DF91893121F4FC
:102D500088277F01A42F0895A993B99343955A9585
:102D6000503019F371917032E9F37C3229F33197C5
:102D7000A42F7F01CF91DF910895A3E0CCDFA33092
:102D800009F590915801B0915A01A0915C01089504
:102D9000D0915801C0915A01F0915C01E0915E011F
:102DA000C0934601D0934901E0934701F0934A0153
:102DB0000895A2E0B1DFA23029F4B0915801A091AA
:102DC0005A010895AF91AF9106C8A2E0A5DFA230E5
:102DD000C9F7C0915801D0915901A0915A01B09101
:102DE0005B010895F70115D0713478F07B3538F424
:102DF0007154770FDCE0C0E9C70FD21D089571361A
:102E000020F07B3710F47156F4CF8F918F9187E0CB
:102E1000089571917032E9F30895F7010895F7016B
:102E20000C946D09EF93FF930E949E31EC2FFD2FC0
:102E300000E00E943E3170912D01713011F4872F16
:102E400008C04A3EC9F400937401003031F4AA2747
:102E5000BB278827FF91EF910895C8E7D1E0A191A2
:102E6000A9930A95E1F7A0E2A993AFEFA993E8E748
:102E7000F1E00E946D09EDCF4C3E49F40030C9F2FB
:102E8000AA940E949E31A0E2A8830A95D2CF403234
:102E900048F24B3738F6AA2DAD3120F60E943D2D71
:102EA0000395C7CF92E0BB27AC2DA3950E94662C5B
:102EB0004AE30E943D2DBB27AD2D0E94662C0E9447
:102EC0003C2D0895DF93CF93BF93AF93A09158010A
:102ED000B0915901B33098F4CCE3DDE0CA0FDB1FA9
:102EE000AF91BF91A883C0915801D091590121960B
:102EF000C0935801D0935901CF91DF910895B450F8
:102F000090F0AA0FBB1FB33070F4CCE3DDE0CA0F22
:102F1000DB1FAF91BF91A993B993C0915801D09194
:102F200059012296E5CF82E1AF91BF91CF91DF9118
:102F3000089570912C01A0FF0895A33059F4509189
:102F40005C015F70550F707F572B70912C0150936F
:102F50002C01089550916001F4CF0E940E20403062
:102F600011F466270895409360010E94FF1F4130CD
:102F700009F066270895AF3F31F42C9A2CBCACE5DC
:102F8000ACBD3DBC08952CBCAF73A064ACBD3DBCD2
:102F90002C980895BDB5B7FFFDCF089550917201EB
:102FA00040917301433038F4DDE0CCE3C50FD41F0A
:102FB000A991BB2710C05050444058F0550F441FF2
:102FC000433038F4DDE0CCE3C50FD41FA991B991AB
:102FD00002C082E108954091720150917301430D46
:102FE000521D4093720150937301803009F408958B
:102FF0004F914F910895A0EAB1E04FEF52E24D9307
:103000005A95E9F7C8E9D1E040E25A91503211F4FB
:103010004A95D9F7442EA0EAB1E0C8E7D1E04C0EBA
:10302000A03C28F4C41518F44881403009F40895F0
:1030300093D04F3FE1F37AD04F3FC9F3403081F74F
:1030400098D0403069F73DD0403051F70AD0403039
:1030500039F74991413618F04B3708F440524D93F7
:10306000DFCF4881403320F04A3310F4405302C090
:1030700044270895642F772721964881403380F0B4
:103080004A3370F44053660F771F0B01660F771FAA
:10309000660F771F600D711D640F721D2196EDCFB5
:1030A000703029F04DE14D937D936D9308956A3012
:1030B00020F04CE14D936D930895605D6D934CE16C
:1030C00008954881443211F04427089566277727F0
:1030D000219658815033F8F05A3310F450530BC0F6
:1030E0005134C8F0573410F4575305C0513698F096
:1030F000573688F457555F705295550F661F771FE6
:10310000550F661F771F550F661F771F550F661FD8
:10311000771F2196DECF703029F04FE14D937D93DC
:103120006D9308954EE14D936D9308954881423219
:1031300011F04427089521964D934991423219F494
:103140004D9341E00895403029F442E24D934FEF12
:103150004D9308954D93F1CF4881473211F04427A4
:10316000089521964D9349914030E1F74FEF4D93EB
:103170000895FF93EF93BF93AF935F93E6E7F4E473
:103180000E014591403089F0689457E0A591AE3228
:1031900039F0B991B13608F0B052AB1709F0E894A4
:1031A0005A95A1F716F0E001EBCF5F91AF91BF9177
:1031B000EF91FF91403041F04D934F934881403261
:1031C00011F42196FBCF4F910895CBE7D1E0A0EA0F
:1031D000B1E040E2E0E24993EA95E9F7A097A03C2C
:1031E00029F04D91423010F04F3F11F4299208958B
:1031F000403220F0403810F486D0F1CF4C3121F429
:10320000ED91FF2719D0EBCF4D3121F4FD91ED91D8
:1032100013D0E5CF4E3131F444E275D0ED91FF2764
:103220003CD0DDCF4F3131F444E26DD0FD91ED91D2
:1032300034D0D5CF50D0D3CFE8944FE24395E0516E
:10324000F742E0F7E05FF84D403311F063D0689447
:103250004FE24395E85EF340E0F7E851FC4F16F08B
:10326000403311F057D068944FE24395E456F04054
:10327000E0F7EC59FF4F16F0403311F04BD0689453
:103280004FE24395EA50E8F7E65F16F0403309F065
:1032900041D040E34E0F3ED00895E8944F2F429521
:1032A0004F7011F012D068944F2F4F700EF011F044
:1032B0000CD068944E2F42954F700EF011F005D04F
:1032C00068944E2F4F7001D00895405D4A3308F046
:1032D000495F20D00895E6E7F4E45591503009F4B1
:1032E0000895451711F03796F8CF5F9357E0459151
:1032F0004E3209F00FD05A95D1F75F915C3110F042
:1033000040E208D008954993CB3918F029924F91A3
:103310004F9108954993CB3928F029924F914F91BD
:103320004F914F910895FF93EF93A0913E01A09389
:103330006E01AA270E94F62BA0912C01A0936A018E
:10334000A0910F01A0936D01A0912A01A0936901A2
:1033500020922A01E8ECF1E0CCE2D7E0BEE2AEE157
:1033600041914993AA95E1F7BA95C9F7EF91FF9179
:103370000895FF93EF93A0916E010E94F62BA09108
:103380006D01A0930F01A0916A01A0932C01A0915F
:103390006901A0932A01ECE2F7E0C8ECD1E0DECFAE
:1033A000A0910C01A4FD35C0C6E0D4E0A9E4BFE4BF
:1033B00041B158E040FDB99340FFA99346955A9515
:1033C000C9F7C4E2D4E0A0E3B1E340B158E040FD66
:1033D000B99340FFA99346955A95C9F7C8EBD6E033
:1033E000AFEABFE241B158E040FDB99340FFA99375
:1033F00046955A95C9F7C6EDD6E0A0E8BEE440B1BF
:1034000058E040FDB99340FFA99346955A95C9F7F6
:1034100008950E94CB2E130020494F204449534168
:10342000424C454420000895452FA6E10E94472CB8
:103430004F5B0E943D2D4DE30E943D2DA7E10E9470
:10344000472CC0E9DCE0C50FD21DC50FD21DA991E4
:10345000B9919DE00E94662C0895A3E10E94E42E9C
:10346000A5E0C62FCA95AC9FCCEEDCE0C00DD11D07
:10347000A881A7FF0AC00E94CB2EFF43414C4C20DD
:103480002000A981AF770EC008950E94CB2EFF4681
:103490004F5220004A8146954F5B0E943D2D0E946D
:1034A0003C2DA981BB27A39592E00E94662C4AE39C
:1034B0000E943D2DBB27A8810E94662C0895209272
:1034C0000F01A7E00E94472C0E94D62C0E94CB2E11
:1034D000120042495420303132333435363700003F
:1034E0000E94CB2E1300444952000E94CB2E1400A0
:1034F0004C455600A7E20E94472C0E94CB2E160096
:103500002045786974200000A0E60E94472C0E94A4
:10351000CB2E16062020476F20200000A0E40E943A
:10352000472C0E94CB2E160C20537465702000008F
:10353000A7E10E94472C0E94CB2E161220566965E7
:1035400077200000AEE6A0932B07A7E30E94472C4C
:103550000E94CB2E1618202020202000A5E00E94DB
:10356000472C0E94CB2E00004156522D43686970B3
:10357000426173696332204D4F4E2020202050005D
:10358000409137014F5C0E943D2D0E94CB2EFF3AA7
:10359000000092E0BB27AC2DA3950E94662C0E94F0
:1035A000CB2EFF3A0000BB27AD2DA3950E94662CC1
:1035B000EBE7F1E0C6EED1E0AEE141EFB191B03022
:1035C00031F0BE8F4CAF4993AA95C1F706C0B0E267
:1035D000BE8F4CAF4993AA95D1F7A7E10E94472C23
:1035E000C0E0D4E0E1E1F0E10E94D02F9DE050E0A6
:1035F000452F4C5FB42FAA270E94E42E15DF539568
:103600005D30B1F7452F4950B42FA9E00E94E42E58
:103610000BDF53955A31B1F7A7E30E94472CC3E162
:10362000D4E0EDE1F0E10E94D02F0E94CB2E0413F4
:10363000535441434B3A00009927BB27A0916F0197
:103640000E94662C6CE0C0916F01C61720F0C61B6B
:10365000B4E0B60F02DF6A95B1F708954F935F9318
:103660006F937F93EF93FF93CF93DF93AF93BF93CA
:10367000AF92BF928F939F9356DEA7DD20DF2ED0AF
:103680008827A0912D014D3E11F4A16011C0413F4A
:1036900011F4AA270DC0423F11F4A46009C0433FB2
:1036A00071F767DE0E943231AA270E94F62BE6CF1F
:1036B000A0932D01409116014030E1F75ADE9F9111
:1036C0008F91BF90AF90BF91AF91DF91CF91FF915C
:1036D000EF917F916F915F914F9108952092170123
:1036E0005FDE409117014030D9F30C94D63120921F
:1036F0002A0120923E01A5E00E94472CC0E0D0E0C4
:10370000EDE1F6E10E946E30A0E50E94472C0E9498
:10371000CB2E010244464C4153482073697A653AE6
:1037200020000E940E204F3749F40E94CB2EFF3517
:103730003132204B69427974650011C04F3F41F42A
:103740000E94CB2EFF31204D69427974650007C07D
:103750000E94CB2EFF3020427974650013C00E9476
:10376000FF1F4130D1F0EAE8F9E3E8940E94F93212
:10377000413009F434C0443009F4B9CF423099F7EC
:1037800033D0B5CFE6ECF9E3E8940E94F93241304A
:1037900009F425C04430B1F7AACFEEE4F9E3E89488
:1037A0000E94F932413009F41AC0473019F40E94DE
:1037B000011D9DCF4A3011F417D099CF423011F43A
:1037C0006DD095CF433019F40E94581D90CF4430EE
:1037D00019F40E94AA1D8BCF4530F9F688CFA0912D
:1037E0001601A030E1F708950E94A8354F466F7288
:1037F0006D6174204D656469756D3F00413009F05D
:103800000895A6E20E94472CC2E0D8E0EBE1FCE07C
:103810000E9436300E94CB2E0903466F726D617490
:1038200074696E672E2E2E202020202020000E94FA
:10383000CB2E0B0300000E941120803001F50E9466
:10384000CB2E0903466F726D617474696E672E2EFC
:103850002E20446F6E652100A2E70E94472C0E9433
:10386000CB2E0B03202020507265737320616E797C
:10387000206B6579212020000E94323108950E943A
:10388000CB2E0903466F726D617474696E672E2EBC
:103890002E204572726F72210000DECFA0E60E94DA
:1038A000472CC4E0D8E0E9E1FDE00E9436300E94F8
:1038B000CB2E0905417661696C61626C653A000046
:1038C0000E94CB2E0A0546696C65733A20009CE085
:1038D0000E94F11FDF93CF93DF010E94662C0E94AC
:1038E000CB2EFF202F000E940E20A42FB0E01196B7
:1038F0000E94662C0E94CB2E0B05426C6F636B738B
:103900003A00AF91BF910E94662C0E94CB2EFF20FF
:103910002F000E94F91FA0EFA49FD0011197B03093
:1039200009F413970E94662CA6E00E94472C0E947F
:10393000CB2E0C05202020507265737320616E79A8
:10394000206B6579212020000E94323108952045A6
:103950007869742020496E666F204261636B7570D0
:10396000526573746F7252657363616E20202020FC
:10397000202044656C6574652020202020202020B4
:1039800020202020466F726D617420457869742074
:10399000466F726D6174202020202020202020207E
:1039A000202052657363616E20202020202020207B
:1039B0002020202020202020202020202020202007
:1039C00020202020202020457869742020202020DD
:1039D0002020202020202020202020202020526570
:1039E0007363616E202020202020202020202020B2
:1039F00020202020202020202020202020202020C7
:103A0000202077270BD1A4E00E94472CC1E0D2E010
:103A1000ECE1F5E10E946E30A0E40E94472C0E9488
:103A2000CB2E030244656C6574652066696C650085
:103A3000B0D070935801D8D24C3FD1F34CD1413023
:103A400019F4A72F8AD2E1D208957727E7D0A4E00E
:103A50000E94472CC1E0D2E0ECE1F5E10E946E301B
:103A6000A0E40E94472CA0E1A0935C010E94CB2E11
:103A7000030253617665205000009AD28AD0709379
:103A80005801B2D2403E20F4403161F0F4D0DECF94
:103A9000A8D2D03021F4CC3010F427D1D7CF5DD2CA
:103AA000B4D108950CD1413089F657D2BAD10895D6
:103AB0007727B4D0A4E00E94472CC1E0D2E0ECE12B
:103AC000F5E10E946E30A0E40E94472CA2E1A09391
:103AD0005C010E94CB2E03024261636B7570000093
:103AE00058D07093580180D2403920F4423161F0AF
:103AF000C2D0DFCF76D2D03021F4C03610F4F5D06A
:103B0000D8CF2BD2EFD10895DAD0413091F625D21B
:103B1000F5D10895772782D0A4E00E94472CC1E018
:103B2000D2E0ECE1F5E10E946E30A0E40E94472C67
:103B30000E94CB2E03024C6F61642050000038D2EB
:103B400028D07093580150D2403111F0A2D0E3CF69
:103B500088D10895772762D0A4E00E94472CC1E065
:103B6000D2E0ECE1F6E10E946E30A0E40E94472C26
:103B70000E94CB2E0302526573746F72650009D0E8
:103B80007093580131D2423111F08ED0E4CFCED1B2
:103B900008957727B5D00BD10E9432314D3E21F4E4
:103BA0002FD14F914F9108954A3E09F40895403E18
:103BB00019F40FD17727EECF413E21F40AD170914D
:103BC0006001E8CF443E49F4703031F302D17150C6
:103BD000472F4F704F30F1F2DECF453E59F4409100
:103BE0006001471709F4D8CFF4D07395472F4F7071
:103BF00089F2D1CF463E29F4703170F2EAD070518B
:103C0000C9CF473E51F4409160014F3031F04051EF
:103C1000471718F0DED0705FBDCFBECF0E940E20D8
:103C2000403019F44F914F911BC0409360010E94A6
:103C300009310E940931E3D1413019F04F914F9180
:103C400001C008950E947F354F44464C415348209F
:103C50006E6F7420666F726D617474656400089590
:103C60000E947F354F44464C415348206572726F25
:103C70007221000008950E947F354F43616E206ECF
:103C80006F742073617665206F6E207468697300AD
:103C900008950E947F354F4E6F2042415349432083
:103CA00066696C65000008950E947F354F4E6F2055
:103CB0004241434B55502066696C650008950E944F
:103CC000A835C04F76657277726974652066696C35
:103CD000653F000008950E94A8354F44656C6574E7
:103CE000652066696C653F0008950E947F354F4EE0
:103CF0006F207370616365206C65667400000895C1
:103D00005F936F937F93A72FA07FA0936C01A091E7
:103D10006C01AF70AB5FBA2FA4E00E94E42EA6E066
:103D20000E94472CA0916C01BB2795E00E94662C55
:103D30000E943C2DA5E00E94472CA0916C01A0930D
:103D4000580152D1ADD04F3F61F1A0916C01A093C9
:103D5000580140E040935A0142E040935C018827BB
:103D600057D1803091F4CCE3DFE00E943C2D5CE041
:103D70005F934991403808F04EE2403208F440E247
:103D80000E943D2D5F915A9599F7A0916C01A395E2
:103D9000A0936C01AF7009F0BACF7F916F915F91E2
:103DA00008955DE00E943C2D5A95E1F7EECF4F93C8
:103DB0005F93C4E1D5E0472F4F705EE1459FC00D92
:103DC000D11D52EF47E159934A95E9F75F914F9121
:103DD00008954F935F93C4E1D5E0472F4F705EE1A4
:103DE000459FC00DD11D5CE044E059934A95E9F729
:103DF0005AE043E159934A95E9F75F914F9108954D
:103E0000A0911601A030E1F70895709358014CE09D
:103E100040935A0140E140935C01F4D0803009F0B6
:103E20001FCF7093580190913D01E0E0F0E9977049
:103E3000929540EC949FE00DF11D40E04F9300E01F
:103E4000CCE3DFE0159119930A95E1F740935A010D
:103E500042E040935C01DFD04F9143954C3071F7C5
:103E6000089590913D019770E0E0F0E9929540EC63
:103E7000949FE00DF11D40E04F9340935A0142E0C2
:103E800040935C0170935801C3D0CCE3DFE00E9403
:103E90006B7932964F9143954C3071F77894089531
:103EA000403139F40E94CB2EFF4241533A0040E1A9
:103EB0000895423139F40E94CB2EFF4255503A000A
:103EC00042E10895443139F40E94CB2EFF555352FC
:103ED0003A0044E108950E94CB2EFF2D2D2D2D0098
:103EE0004FEF08957093580140E640935A0142E124
:103EF00040935C0187D0803009F0B2CE70935801B6
:103F00004427E0E0F0E94F93CCE3DFE00024159094
:103F100019920A94E1F740935A0142E040935C0100
:103F20007AD04F914395403671F7089540E0E0E034
:103F3000F0E94F9340935A0142E040935C01709343
:103F4000580166D0CCE3DFE00E946B7932964F9146
:103F50004395403671F7789408954F93FF93EF930C
:103F6000DF93CF93BF93AF9340912C0140936101B6
:103F70004CE440932C01C6E0DAE0E7E1FCE00E946B
:103F800036300E94CB2E0B0757726974696E67201A
:103F9000646174612E2E2E004091610140932C01CA
:103FA000AF91BF91CF91DF91EF91FF914F91089524
:103FB000CAE2CAE240913D01942F4F5C499340E22E
:103FC00049934BE54993409129014F9340684093B1
:103FD00029010E949D794DE549934F914093290114
:103FE00008950E94103A08950E94DC3A0E949F387A
:103FF00008950E944C3808950E94CC3808950E947C
:10400000EB3908950E94713A08950E94E43A0895A8
:104010000E94643B08950E94053B08950E945A380F
:1040200008950E947D390895A1E00E94BE32209239
:104030002A0120923E01A7E00E94472CC0E0D0E078
:10404000EDE1F6E10E946E30A0E70E94472C0E944D
:10405000CB2E01024156522D43686970426173694B
:10406000633220636F6E6669677061676500A7E001
:104070000E94472C0E94CB2E1401436865636B732A
:10408000756D3A20000014D144D078D0AAD0DAD08F
:10409000E2E1F3E4E8940E94F932413009F403C10B
:1040A000423059F440910C0151E0452740930C01F6
:1040B0000E9407790E945321E7CF433059F4409181
:1040C0000C0152E0452740930C010E9407790E94A1
:1040D0005321DACF443059F440910C0154E0452784
:1040E00040930C010E9407790E945321CDCF4530A7
:1040F00059F440910C0158E0452740930C010E946F
:1041000007790E945321C0CF4A3011F40E94C2287F
:104110008BCFA6E00E94472C0E94CB2E03014B655B
:1041200079626F617264206C61796F75743A000016
:10413000A7E040910C01417009F4A1E70E94472CCF
:104140000E94CB2E03124445202851574552545A01
:104150002900A7E040910C01417009F0A1E70E94FD
:10416000472C0E94CB2E04125553202851574552FC
:1041700054592900A7E00E94472C0895A6E00E9408
:10418000472C0E94CB2E060153657269616C20702A
:104190006F72743A0000A7E040910C01427009F47C
:1041A000A1E70E94472C0E94CB2E0612203132300C
:1041B0003020427073202000A7E040910C01427033
:1041C00009F0A1E70E94472C0E94CB2E0712203253
:1041D00034303020427073202000A7E00E94472C2A
:1041E0000895A6E00E94472C0E94CB2E0901493277
:1041F0004320706F72743A00A7E040910C01447044
:1042000009F4A1E70E94472C0E94CB2E091220201E
:10421000313030206B487A202000A7E040910C011B
:10422000447009F0A1E70E94472C0E94CB2E0A128D
:104230002020343030206B487A202000A7E00E94F4
:10424000472C0895A6E00E94472C0E94CB2E0C011B
:1042500053504920706F72743A00A7E040910C01EE
:10426000487009F4A1E70E94472C0E94CB2E0C1243
:104270002020202035204D487A202000A7E04091C2
:104280000C01487009F0A1E70E94472C0E94CB2E38
:104290000D122020313536206B487A202000A7E00F
:1042A0000E94472C0895A0911601A030E1F70895CF
:1042B000AA27BB27CC27DD27EE27FF27159042E052
:1042C000149EA00DB11DC21DD21D459147E0149E44
:1042D000A00DB11DC21DD21DFE3881F7EE27F0EFF3
:1042E000459141E7149EB01DC11DD21D459147E087
:1042F000149EB01DC11DD21DF03091F7BF93AF9336
:10430000DE019FE00E94C12CAF91BF910E94C12CA1
:104310000895204578697420204B657962202053E8
:10432000657220202049324320202053504920200C
:10433000202020202020202020202020202020207D
:104340002020202020202020436C6F6E6520AEE0CE
:10435000A0932C01C1E0D4E0ECE1F1E10E94363001
:104360000E94CB2E050500000E94F7010E94CB2E73
:10437000060328632920323030362D38204A6F65F5
:10438000726720576F6C6672616D0000A2EAA0939D
:104390002C010E94CB2E08032020202020204465E1
:1043A0006469636174656420746F2020202020207C
:1043B00000000E94CB2E0903466C6F7269616E2C5F
:1043C000204572696B20616E64204469616E612EC4
:1043D0000000AEE0A0932C010E94CB2E0B0254688B
:1043E000697320736F667477617265206973206CDE
:1043F0006963656E736564000E94CB2E0C04756E54
:1044000064657220746865207465726D73206F66D0
:104410002074686520000E94CB2E0D04474E552065
:104420005055424C4943204C4943454E5345205634
:104430002E3220000E94CB2E0E0355736520697426
:1044400020617420796F7572206F776E20726973A6
:104450006B210000A2ECA0932C010E94CB2E100730
:1044600020505245535320414E59204B455920006E
:104470000E943231089502414253282E2E2E0353BA
:10448000474E282E2E2E04535152282E2E2E054EE6
:104490004F54282E2E2E06524E44282E2E2E0741E3
:1044A0004443282E2E2E08494E282E2E2E2E0958F3
:1044B0005045454B282E0A54454D50282E2E0B4C66
:1044C0004F282E2E2E2E0C4849282E2E2E2E0D4BE8
:1044D0004559282E2E2E0E455045454B282E0F456A
:1044E0005252282E2E2E104152282E2E2E2E11538F
:1044F000494E282E2E2E12434F53282E2E2E134671
:1045000054595045282E144653495A45282E1550C3
:1045100053544154282E16535049282E2E2E174DF1
:10452000454E55282E2E805052494E542E2E8143F2
:104530004C532E2E2E2E82474F544F2E2E2E83421A
:104540004F582E2E2E2E8441434F50592E2E8553D8
:10455000594E432E2E2E86454E442E2E2E2E874209
:10456000434F50592E2E885448454E2E2E2E89509A
:104570004F532E2E2E2E8A4E4F54452E2E2E8B45C7
:104580004D49542E2E2E8C52524541442E2E8D5282
:1045900057524954452E8E474F5355422E2E8F5217
:1045A000455455524E2E90564D4F44452E2E914E09
:1045B0004558542E2E2E92494E5055542E2E93501F
:1045C0004C4F542E2E2E94574149542E2E2E955436
:1045D0005345542E2E2E96544745542E2E2E974634
:1045E00053454C454354984F4E4552522E2E9953A5
:1045F0005055542E2E2E9A534745542E2E2E9B4501
:10460000504F4B452E2E9C4745545049582E9D43A4
:104610004952434C452E9E434F4C4F522E2E9F42A3
:104620004F524445522EA0464F4E542E2E2EA1508E
:10463000554D502E2E2EA258504F4B452E2EA3597D
:10464000454D49542E2EA44C494D49542E2EA54774
:10465000455443484152A644524157544F2EA75007
:104660004C41592E2E2EA85350524954452EA95331
:1046700043524F4C4C2EAA425245414B2E2EAB4634
:104680004153542E2E2EAC534C4F572E2E2EAD444C
:104690005241572E2E2EAE49434F4D4D2E2EAF4434
:1046A0004154412E2E2EB043544558542E2EB1461F
:1046B000524541442E2EB24657524954452EB343DB
:1046C000424F582E2E2EB447455441545452B546AD
:1046D00044454C455445B646424F582E2E2EB750B1
:1046E000414C45545445B8464F522E2E2E2EB949B2
:1046F000462E2E2E2E2EBA4449522E2E2E2EBB4F33
:1047000055542E2E2E2EBC46434952434C45BD4196
:104710004C4552542E2EBE46435245415445BF414E
:10472000534B2E2E2E2EC03F2E2E2E2E2E2EC74217
:10473000432E2E2E2E2ECA4E4F2E2E2E2E2ECB45F3
:104740004D2E2E2E2E2ECC5252442E2E2E2ECD52AB
:1047500057522E2E2E2ECE474F532E2E2E2ECF5268
:1047600045542E2E2E2EC2474F2E2E2E2E2ED05694
:104770004D2E2E2E2E2ED2494E502E2E2E2ED35072
:104780004C2E2E2E2E2ED74653454C2E2E2EDC4749
:1047900050582E2E2E2EDD43492E2E2E2E2EDE4349
:1047A0004F4C2E2E2E2EDF424F2E2E2E2E2EE44C30
:1047B000494D2E2E2E2EE54743482E2E2E2EE64412
:1047C000544F2E2E2E2EE85350522E2E2E2EED44C8
:1047D000522E2E2E2E2EEE49432E2E2E2E2EEF440E
:1047E000412E2E2E2E2EF14652442E2E2E2EF246E5
:1047F00057522E2E2E2EF44741542E2E2E2EF54695
:1048000044454C2E2E2EF750414C2E2E2E2EFC467B
:1048100043492E2E2E2EFE4643522E2E2E2E002E95
:104820002E2E2E2E2E2EA0910801B0910901ED0101
:10483000E2EBF2E0CE0FDF1FF6EFE0910E01FE0F8C
:104840007F934F92EEE14E2E6991ED915491762F28
:104850007295762757FD672768B9ED91000056FDE0
:1048600076B9049055FD76B96991162E54FD76B946
:104870001294162653FD76B907FC61254A9452FD21
:1048800076B9502D712D41F760910F0168B94F90A5
:104890007F91EE91F0910E01F395FA3029F4FF2704
:1048A000A0930801B0930901F0930E010C94F92A2A
:1048B000A0910801B0910901D0910001C0910101BE
:1048C000C295DC0FDE7EE5E110900F01FD914D2FCA
:1048D000F0FD429548B900004D2FF1FD429548B9D1
:1048E00000004D2FF2FD429548B900004D2FF3FD19
:1048F0004295000048B96D2F4D2FF4FD429548B9FF
:10490000CD91F5FD62955D2F68B9F6FD52956D2F3D
:104910004D2F58B9F7FD6295C0FD4295000068B96A
:10492000FC2FEA95B9F618B8EE91F0910E01F395C7
:10493000F23029F4FF27A0930801B0930901F09306
:104940000E010C94F92AA0910801B0910901D1E05F
:10495000FEE110900F01ED91CE2FC370588158B930
:10496000CE2FC695C695C3705881E29558B9CE2F03
:10497000C3705881CE2FC69558B9C695C37058815B
:10498000ED91CE2F58B9C3705881FA9541F718B8F8
:10499000EE91F0910E01F395F33029F4FF27A093E7
:1049A0000801B0930901F0930E010C94F92AA0912B
:1049B0000801B09109010F9310900F01EAE2D1E0D4
:1049C000CD91C6950C2FC295C770F881F8B9C02F4C
:1049D0000000C770F881000000000000F8B9CD9118
:1049E000C6950C2FC295C770F881EA9579F718B86B
:1049F00011970F91F0910E01F395F43029F4FF27F0
:104A0000A0930801B0930901F0930E010C94F92AC8
:104A1000A0910801B0910901D0910001C09101015C
:104A2000C295DC0FDE7EE0E110900F01FD914D2F6D
:104A3000F0FD429548B90000000000004D2FF1FD47
:104A4000429548B90000000000004D2FF2FD42954C
:104A500048B9000000004D2FF3FD4295000048B911
:104A6000000000006D2F4D2FF4FD429548B9000065
:104A7000CD91F5FD62955D2F68B900000000F6FD4F
:104A800052956D2F4D2F58B9F7FD6295C0FD429597
:104A90000000000068B9FC2F00000000EA9551F604
:104AA000000018B8EE91F0910E01F395F33029F45F
:104AB000FF27A0930801B0930901F0930E010C9415
:104AC000F92AA0910801B0910901C0914101D82DA6
:104AD000F6EFE0910E01FE0FE395E0930E01EA3050
:104AE00088F1EC3069F59396A0930801B093090121
:104AF00020920E01DC3031F4D0914001D09341017D
:104B00000C94F92AD83189F4A1E3B2E0C0912E01C6
:104B1000D3E2CD9FA00DB11DCFE0A0930801B093CB
:104B20000901C09341010C94F92AD83D49F4CBE422
:104B3000AEE0B2E0A0930801B0930901C093410137
:104B40000C94F92A0F931F932F93D83D28F4DC2F50
:104B50000C2F1C2F2C2F05C029E61DE208E8DCECE9
:104B6000CBE46C2F7C2F7295ED91E7FD6727EF77F3
:104B70005491ED9168B9172E56FD16B86C2F7C2F05
:104B8000729555FD16B8E7FD672754FD16B8EF7707
:104B9000000053FD16B8049052FD16B8502DED914B
:104BA00068B9172E56FD16B86C2F7C2F729555FDDF
:104BB00016B8E7FD672754FD16B8EF77000053FDE0
:104BC00016B8049052FD16B8502DED9168B9172E05
:104BD00056FD16B86C2F7C2F729555FD16B8E7FD63
:104BE000672754FD16B8EF77000053FD16B8049000
:104BF00052FD16B8502DED9168B9172E56FD16B816
:104C00006C2F7C2F729555FD16B8E7FD672754FD74
:104C100016B8EF77000053FD16B8049052FD16B891
:104C2000502DED9168B9172E56FD16B86C2F7C2FBC
:104C3000729555FD16B8E7FD672754FD16B8EF7756
:104C4000000053FD16B8049052FD16B8502DED919A
:104C500068B9172E56FD16B86C2F7C2F729555FD2E
:104C600016B8E7FD672754FD16B8EF77000053FD2F
:104C700016B8049052FD16B8502DED9168B9172E54
:104C800056FD16B86D2F7D2F729555FD16B8E7FDB0
:104C9000672754FD16B8EF77000053FD16B804904F
:104CA00052FD16B8502DED9168B9172E56FD16B865
:104CB0006D2F7D2F729555FD16B8E7FD672754FDC2
:104CC00016B8EF77000053FD16B8049052FD16B8E1
:104CD000502DED9168B9172E56FD16B86D2F7D2F0A
:104CE000729555FD16B8E7FD672754FD16B8EF77A6
:104CF000000053FD16B8049052FD16B8502DED91EA
:104D000068B9172E56FD16B86D2F7D2F729555FD7B
:104D100016B8E7FD672754FD16B8EF77000053FD7E
:104D200016B8049052FD16B8502DED9168B9172EA3
:104D300056FD16B86D2F7D2F729555FD16B8E7FDFF
:104D4000672754FD16B8EF77000053FD16B804909E
:104D500052FD16B8502DED9168B9172E56FD16B8B4
:104D60006D2F7D2F729555FD16B8E7FD672754FD11
:104D700016B8EF77000053FD16B8049052FD16B830
:104D8000502DED9168B9172E56FD16B86D2F7D2F59
:104D9000729555FD16B8E7FD672754FD16B8EF77F5
:104DA000000053FD16B8049052FD16B8502DED9139
:104DB00068B9172E56FD16B8602F702F729555FDE5
:104DC00016B8E7FD672754FD16B8EF77000053FDCE
:104DD00016B8049052FD16B8502DED9168B9172EF3
:104DE00056FD16B8602F702F729555FD16B8E7FD69
:104DF000672754FD16B8EF77000053FD16B80490EE
:104E000052FD16B8502DED9168B9172E56FD16B803
:104E1000602F702F729555FD16B8E7FD672754FD7A
:104E200016B8EF77000053FD16B8049052FD16B87F
:104E3000502DED9168B9172E56FD16B8602F702FC2
:104E4000729555FD16B8E7FD672754FD16B8EF7744
:104E5000000053FD16B8049052FD16B8502DED9188
:104E600068B9172E56FD16B8602F702F729555FD34
:104E700016B8E7FD672754FD16B8EF77000053FD1D
:104E800016B8049052FD16B8502DED9168B9172E42
:104E900056FD16B8602F702F729555FD16B8E7FDB8
:104EA000672754FD16B8EF77000053FD16B804903D
:104EB00052FD16B8502DED9168B9172E56FD16B853
:104EC000612F712F729555FD16B8E7FD672754FDC8
:104ED00016B8EF77000053FD16B8049052FD16B8CF
:104EE000502DED9168B9172E56FD16B8612F712F10
:104EF000729555FD16B8E7FD672754FD16B8EF7794
:104F0000000053FD16B8049052FD16B8502DED91D7
:104F100068B9172E56FD16B8612F712F729555FD81
:104F200016B8E7FD672754FD16B8EF77000053FD6C
:104F300016B8049052FD16B8502DED9168B9172E91
:104F400056FD16B8612F712F729555FD16B8E7FD05
:104F5000672754FD16B8EF77000053FD16B804908C
:104F600052FD16B8502DED9168B9172E56FD16B8A2
:104F7000612F712F729555FD16B8E7FD672754FD17
:104F800016B8EF77000053FD16B8049052FD16B81E
:104F9000502DED9168B9172E56FD16B8612F712F5F
:104FA000729555FD16B8E7FD672754FD16B8EF77E3
:104FB000000053FD16B8049052FD16B8502DED9127
:104FC00068B9172E56FD16B8612F712F729555FDD1
:104FD00016B8E7FD672754FD16B8EF77000053FDBC
:104FE00016B8049052FD16B8502DED9168B9172EE1
:104FF00056FD16B8612F712F729555FD16B8E7FD55
:10500000672754FD16B8EF77000053FD16B80490DB
:1050100052FD16B8502DED9168B9172E56FD16B8F1
:10502000622F722F729555FD16B8E7FD672754FD64
:1050300016B8EF77000053FD16B8049052FD16B86D
:10504000502DED9168B9172E56FD16B8622F722FAC
:10505000729555FD16B8E7FD672754FD16B8EF7732
:10506000000053FD16B8049052FD16B8502DED9176
:1050700068B9172E56FD16B8622F722F729555FD1E
:1050800016B8E7FD672754FD16B8EF77000053FD0B
:1050900016B8049052FD16B8502DED9168B9172E30
:1050A00056FD16B8622F722F729555FD16B8E7FDA2
:1050B000672754FD16B8EF77000053FD16B804902B
:1050C00052FD16B8502DED9168B9172E56FD16B841
:1050D000622F722F729555FD16B8E7FD672754FDB4
:1050E00016B8EF77000053FD16B8049052FD16B8BD
:1050F000502DED9168B9172E56FD16B8622F722FFC
:10510000729555FD16B8E7FD672754FD16B8EF7781
:10511000000053FD16B8049052FD16B8502DED91C5
:1051200068B9172E56FD16B8622F722F729555FD6D
:1051300016B8E7FD672754FD16B8EF77000053FD5A
:1051400016B8049052FD16B8502DED9168B9172E7F
:1051500056FD16B8622F722F729555FD16B8E7FDF1
:10516000672754FD16B8EF77000053FD16B804907A
:1051700052FD16B8502DED9128B82F911F910F9127
:105180000C94F92A0E94A8356F436C6F6E652073EA
:10519000797374656D3F2000413009F0089565D042
:1051A00087D0803079F078D00E947F354F4E6F20C5
:1051B000636F6E74726F6C6C657220666F756E646F
:1051C000200008958DD0803069F066D00E947F3530
:1051D0004F4E6F204D65676136343420666F756EB3
:1051E00064000895CBD09BD0EE27FF2750E060E00D
:1051F0000590B6D00590BBD063956038C9F79CD0B8
:105200005395A9F74CEA4ED040EA4CD04AD046EE2E
:1052100049D00E9409310E9409310E9409314CEAAB
:1052200041D048EA3FD03DD041ED3CD00E94093109
:105230000E9409310E9409314CEA34D044EA32D04C
:1052400030D04CEF2FD00E9409310E9409310E94CA
:10525000093122D00E947F358053797374656D20A7
:10526000636C6F6E65640000089543E54CBD2DBC12
:10527000249A2C984FEF4A95F1F72C9A4FEF4A95C4
:10528000F1F72C984FEF4A95F1F72C984FEF4A958C
:10529000F1F70E94093108952C9A4CE54CBD3DBCB4
:1052A000089544274EBD4DB547FFFDCF4EB5089537
:1052B00088274CEAF7DF43E5F5DFF3DF433509F0F4
:1052C00081E0EFDF0895BF93AF934F93A42FBB27E7
:1052D0000E94C12C0E943C2D4F91AF91BF91089527
:1052E000882740E3DFDFDDDF40E0DCDFDADF4E315F
:1052F00011F082E0089540E3D5DFD3DF41E0D2DF53
:10530000D0DF463911F082E0089540E3CBDFC9DFFA
:1053100042E0C8DFC6DF493009F082E008954CEA78
:10532000C1DF40E8BFDFBDDFBCDF0E9409310E9462
:1053300009310E94093108954CE4B4DF452F4695A8
:10534000B1DF452F440F440F440F440F440F440F67
:10535000440FA8DFA6DF0E9409310E940931089599
:1053600040E4A0DF9EDF462F9DDF402D9BCF48E429
:1053700099DF97DF462F96DF402D94CF4F93FF9311
:10538000EF93DF93CF93BF93AF9340912C01409362
:1053900061014CE440932C01C5E0DAE0E8E1FCE077
:1053A0000E9436300E94CB2E0B06436C6F6E696EE6
:1053B000672053797374656D2E2E2E004091610124
:1053C00040932C01AF91BF91CF91DF91EF91FF916D
:1053D0004F91089528B818954F935F936F93FF935B
:1053E000EF93DF93CF93BF93AF930F921F92FFB7CB
:1053F000FF9330921101B0913101B7FF5C98B7FD76
:105400005C9A4B99BE7F4B9BB160B0933101C8E071
:10541000D1E05F89A889E9890A881B88A00DE11D70
:10542000A88BE98BFFA14491AD89AF3F09F4452FCB
:105430005AA54503B0E8B10DB093B300EE89FF89DA
:10544000488D598DAA27E2FDA095E5FDA095F4FDB4
:10545000A09557FDA095AA1FEE1FFF1F441F551FC3
:10546000EE8BFF8B488F598F830C921CEBA9FF8129
:10547000EF23E8B97894E9A190FC04C0F8A58F1651
:1054800008F490C0FCE0E2FFFDEE8F1639F45E9860
:10549000E3FFAFC0B2E8B0938000ABC0F1E1E2FF40
:1054A000F3EF8F1639F45E9AE3FFA3C0B2ECB0932A
:1054B00080009FC0FBE1E2FFFFEF8F1621F4EFEFCA
:1054C000E0933B0196C0F2E0E2FFF9EE8F1619F48B
:1054D00020923B018EC0F9E3E2FFF7E08F1609F05E
:1054E00088C0A8ECA883A1E0A9832E8288249924EF
:1054F000AAE0A9AFA5E0E2FFA39542E3E2FF4CE3F7
:10550000BA8DB395BA1731F4BB27EB8DFC8D31966C
:10551000EB8FFC8FBA8FE885E395E41709F4EE274B
:10552000E887FDE8E0E0AC89EA0FF21DB491B2151E
:1055300011F0A395AC8BBAA7A0915001A03009F44B
:1055400058C0B0915101B395B0935101BA17C0F34F
:10555000BB27B0935101E0915201F0915301C091EA
:105560005601D09157012196A191E0935201F093F9
:105570005301AE3F09F056D6FD1798F0EC1788F0AE
:10558000A0913301A13029F4A2E020925001A09310
:105590003301E0915401F0915501E0935201F093F1
:1055A000530127C0A0918400AA3FE0F3AB3F00F075
:1055B000AC3F00F0AD3F00F0AE3F00F0E5FD19C09C
:1055C000E0912901E7FD0C946125E0913E01E53071
:1055D00011F40C940825E37011F40C941324E130B9
:1055E00011F40C945824E23011F40C94A3240C947C
:1055F000D724A0911401A5FD23C0E091C000E7FFCE
:1056000065C0E091C600F5EFB491B0FF34C0A7FFCC
:1056100003C02092160157C0E33809F4E0E1F6E830
:1056200040910C0140FDF395EF77A4FFA6FDF395A3
:10563000A4FFA0FDE068E491E0931501A06244C0DE
:10564000E0911501E0931601E0931701EE3E19F485
:10565000A2FD0C94380040912D01E33611F4A2FD17
:105660004160E03711F4A2FD4260EC3F09F4446070
:1056700040932D0128C0E03F11F4A06825C0E03E12
:1056800011F4A06421C0E23121F4A160A7FDAE7F36
:105690001AC0E93521F4A260A7FDAD7F14C0E43142
:1056A00051F4A6FD04C0A460A7FDAB7F0CC0A860A8
:1056B000A7FDA77F08C0E13121F4A061A7FDAF7E5F
:1056C00002C020921601AF71A093140140910C0109
:1056D00041FD0E94A17841FF0E94D678FF91FFBF53
:1056E0001F900F90AF91BF91CF91DF91EF91FF91FC
:1056F0006F915F914F911895AAEBA4B9AFEFA5B93F
:10570000A0EEA7B9A0E0A8B9A0EFAAB9AFEFABB9D6
:10571000A6B1AF77A0932901B2ECB0938000B9E1B4
:10572000B0938100F4E0A2FFF4E0F0938700FEEF75
:10573000A2FFF6EFF093860020928900FAE5F0933D
:105740008800F4E0F0938B00F8EDF0938A00A6E077
:10575000A0936F00A2E0A4BDA1E0A5BDA1E3A7BDF9
:10576000A3E8A093B000A1E0A093B100A0E8A093AB
:10577000B3002092B6002092C000A0E1A093C10027
:10578000A6E6A093C200ACE5B0910C01B3FDAFE575
:10579000ACBDA0E0ADBDA5E17AD0C8E0D1E0A8ECF9
:1057A000A993A1E0A993AEE12992AA95E9F7AAEA03
:1057B000A0931E01A093200120922A0120920D01A6
:1057C000AEE3A0931C010F93009129010F77009382
:1057D000290106EE07C00F9300912901006800938C
:1057E000290104EE009330010F910895A0933E012A
:1057F000A03041F4ACE3A0934401AEE2A093450194
:10580000A6EE42C0A13069F4A8EAA0934401A4E73F
:10581000A0934501A0E0A0930001A0EEA093010198
:1058200024C0A23091F4A8E7A0934401ACE4A09373
:105830004501C0E0D1E0A0E0A993A0E4A993A0EACB
:10584000A993A0EEA993A3EE1FC0A33081F4A4E511
:10585000A0934401AAE3A0934501C0E0D1E0AA27A8
:10586000B8E0A993A05EBA95E1F7A7EE0DC0A0E855
:10587000A0934401A0E4A0934501A0E2A0930001FD
:10588000A0EEA0930101A0ECA09330010895AA0F0F
:10589000AE7EA0932C010895A295AA0FA07EA0939E
:1058A0000F01089548834091290147FD0EC0CF9311
:1058B000DF935F9342EBC40F42E0D41F40912C0171
:1058C0004E7E48835F91DF91CF9108954F935F9310
:1058D0006F93AF93BF9340E2592F5370523061F0F2
:1058E000533009F44BE2B7FF05C0A095B095A30D66
:1058F000B21D4DE20E943D2D592F5C70692F6073DF
:10590000E8944FE24395A051B742E0F7A05FB84D4D
:105910005C3009F42BD04FE24395A85EB340E0F72A
:10592000A851BC4F53FD22D0603309F4A3D04FE2FD
:105930004395A456B209E0F7AC59BF4F503009F077
:1059400015D0603209F496D04FE24395AA50E8F79B
:105950000DD0A65F603109F48DD040E34A0F8DD0A1
:10596000BF91AF916F915F914F910895403311F0C6
:10597000689483C091FD81C0F6F390FF08957CC0C8
:1059800008954F9390FF05C04B2F429509D04B2FA0
:1059900007D04A2F429504D04A2F02D04F91089544
:1059A0004F70405D4A3308F0495F67C040913E0147
:1059B0004030B1F0AF93BF93CF93DF93D1E0C8EC09
:1059C000ACE5BEE12992BA95E9F7AA95D1F7DF9146
:1059D000CF91AA24BB2420922B01BF91AF910895AF
:1059E000AF93BF93CF93DF93D1E0C8ECA7E1BEE1C3
:1059F0004993BA95E9F7AA95D1F740912C014E7ECB
:105A0000A7E1BEE14993BA95E9F7AA95D1F7DF91ED
:105A1000CF91AA24BB2420922B01BF91AF9108956E
:105A2000AF93BF9320922B01A0912A01A03051F493
:105A3000A7E1AA24B394AB1571F7B6E1BB2ECF93BF
:105A4000DF9362C0A13029F4BF91AF914AE00C947A
:105A5000C632A23021F4BF91AF914AE090C4A33086
:105A600019F4BF91AF910895BF91AF915AE00E9490
:105A7000873708954CE201C040E2AF93BF93A091F5
:105A80002B01A395A0932B01A0912A01A43030F003
:105A9000BF91AF91542F0E9487370895A030A9F08D
:105AA000A33059F4A42FBB275F936F930E94621712
:105AB0006F915F91BF91AF910895BF91AF91A09108
:105AC0002A01A1FF0C94C6325AC4EF93E0913E0123
:105AD000E03009F09AC0EF91CF93DF932FD496FD79
:105AE00035C0E0DEA395AE3131F4AA27B395B731C6
:105AF00011F4B6E107C0AA2EBB2EDF91CF91BF9162
:105B0000AF910895AA2EBB2ED1E0C8EC4F93A6E129
:105B1000BEE14E8D4993BA95E1F7AA95C9F7AEE17A
:105B200040E24993AA95E9F7D4E0CAE7A6E1BEE1CD
:105B30004E8D4993BA95E1F7AA95C9F7AEE1409128
:105B40002C014993AA95E9F74F91D7CFAB31A8F62D
:105B5000B23198F6AD5FAA2EEF93FF934F925F920A
:105B60006F927F9270F85F93E42FF6EFB5E04424D4
:105B7000552466245527A491A7FD539550FB40F862
:105B8000A6FD539550FB41F8A5FD539550FB50F8E9
:105B9000A4FD539550FB51F8A3FD539550FB60F8BD
:105BA000A2FD539550FB61F8F3955527A491A7FDED
:105BB000539550FB42F8A6FD539550FB43F8A5FDC5
:105BC000539550FB52F8A4FD539550FB53F8A3FD99
:105BD000539550FB62F8A2FD539550FB63F8F39583
:105BE000442D60DE2196452D5DDE2196462D5ADE40
:105BF0006C96BA9509F0BBCF5F9170FA7F906F9069
:105C00005F904F90FF91EF9178CFFF93CF93DF9309
:105C10006F937F93E42F60910D0160FD1EC0F6EF3E
:105C2000AA2DBB2DDAE0C49137D0B395AA2D96FDED
:105C300033D096FDB395F395AA2DDA95A1F7AA2D49
:105C4000AA5F96FDAA5FAA2E7F916F91DF91CF91F7
:105C5000FF91EF91BF91AF910895F7E7EF77AE2FE6
:105C6000ECE7EA0FF21DAA0FEA0FF21DAA2DBB2DD9
:105C7000D6E0C49155D0B395AA2D96FD51D096FD8E
:105C8000B395D0FD3196AA2DDA9599F7AA2DAC5F80
:105C900096FDAC5FAA2ED8CF60912C016F936295D0
:105CA000C7FD629560932C01A2D0A39596FD9FD06D
:105CB00096FDA395C6FD629560932C0198D0A3959F
:105CC00096FD95D096FDA395C5FD629560932C0138
:105CD0008ED0A39596FD8BD096FDA395C4FD6295BD
:105CE00060932C0184D0A39596FD81D096FDA39559
:105CF000C3FD629560932C017AD0A39596FD77D071
:105D000096FDA395C2FD629560932C0170D0A3957A
:105D100096FD6DD096FDA3956F9160932C0108952B
:105D200060912C01D0FDC295762FC7FF72957093BC
:105D30002C015DD0A39596FD5AD096FDA395762FA4
:105D4000C6FF729570932C0152D0A39596FD4FD04B
:105D500096FDA395762FC5FF729570932C0147D0C1
:105D6000A39596FD44D096FDA395762FC4FF72951A
:105D700070932C013CD0A39596FD39D096FDA39548
:105D800060932C0108954F934591403011F44F9149
:105D9000089573DEF9CFFF91EF91EE0FFF1FAF93E0
:105DA000BF93B591BF3F11F0A5910ED0BF91AF91B8
:105DB0004F934591403031F44F913197F695E795E7
:105DC000319609945ADEF5CFEF93E0913E01E03031
:105DD00021F0EF91AA2EBB2E0895EF91AE3108F07D
:105DE000ADE1B73108F0B6E1AA2EBB2E0895CF93EE
:105DF000DF93C0914401CA1728F0C0914501CB1729
:105E000008F003C0DF91CF910895AF93BF934F93F4
:105E10005F93C0913E01C53021F0C37031F0C230B4
:105E200008F441C009F464C081C051E0AC3360F5AE
:105E3000BE3250F5B0FD550FB0FD550FA0FD550F0A
:105E4000B695A695CEE1BC9FD1E0C8ECCA0FD21D95
:105E5000C00DD11DA2EBB2E0CA0FDB1FA881B0912B
:105E60002C01BE70B295A07EBA17A9F0B0912C019A
:105E7000BE70AB2BAE7EA883A2EBB2E0CA1BDB0BDD
:105E8000B881B52BBF70B8835F914F91BF91AF912F
:105E9000DF91CF910895A2EBB2E0CA1BDB0BB88172
:105EA0005095B523EFCFCA2FC770C39540E0089433
:105EB000441FCA95E9F7A695A695A695C5E1D09188
:105EC0003E01D2FDC0E1BC9FD1E0C8ECCA0FD21D9B
:105ED000C00DD11DA0912C01A695A17029F440956B
:105EE000A881A423A883D0CFA881A42BA883CCCF3A
:105EF000CA2F50912C015695537043E0C37031F076
:105F0000440F440F550F550FCA95C9F74095A695F4
:105F1000A695CEE1BC9FD1E0C8ECCA0FD21DC00D42
:105F2000D11DA881A423A52BA883AECFCA2F509141
:105F30002C015E704EE0C17011F44295529540956F
:105F4000A695CAE2BC9FD1E0C8ECCA0FD21DC00D15
:105F5000D11DA881A423A52BA88396CFCE3108F00C
:105F6000CDE1EE3108F0EDE1D73108F0D6E1F731BF
:105F700008F0F6E1EC1718F40E2EEC2FC02DFD17EB
:105F800018F40F2EFD2FD02D0895EC1718F40E2EB7
:105F9000EC2FC02DFD1718F40F2EFD2FD02D0895D6
:105FA000AF93BF93CF93DF93EF93FF935F93D6DFCE
:105FB000AC2FBD2FCF93DF93C3D1288252EBC50FF7
:105FC00052E0D51F50912C015883DF91CF91AE172D
:105FD00011F0A395EFCFBF1719F0AC2FB395EACF0F
:105FE0005F91FF91EF91DF91CF91BF91AF910895B4
:105FF000AF93BF93CF93DF93EF93FF935F93C5DF8F
:10600000AC2FBD2FF4DEA395AE17E1F7F0DEB3950C
:10601000FB17E1F7ECDEAA95AC17E1F7E8DEBA95DD
:10602000BD17E1F75F91FF91EF91DF91CF91BF91A4
:10603000AF910895AF93BF93CF93DF93EF93FF9307
:106040005F93A3DFBD2FAC2FD2DEAE1711F0A39567
:10605000FBCFCDDEFB1711F0B395F5CF5F91FF912C
:10606000EF91DF91CF91BF91AF91089599DFAF93F9
:10607000BF93CF93DF93EF93FF934F935F936EDFC5
:106080004C2FBD2FAC2F5CD152EF599351EFA395FC
:10609000AE1711F05993FBCF53EF5993A42FB3953B
:1060A000BF1739F04DD150EF5993AE2F49D15993C5
:1060B000F5CFA42F45D154EF599351EFA395AE17C7
:1060C00011F05993FBCF55EF59935F914F91FF9189
:1060D000EF91DF91CF91BF91AF910895C7DF5F93AB
:1060E000AF93BF93CF93DF93EF93FF9337DFBD2F32
:1060F000AC2F26D15BEF59935CEEA395AE1711F050
:106100005993FBCF5CEF5993FF91EF91DF91CF91C2
:10611000CF93DF93EF93FF93BD2FAC2FB39510D1A7
:106120005DEF599350E2A395AE1711F05993FBCF51
:106130005EEF5993FF91EF91DF91CF91CF93DF9372
:10614000EF93FF93BD2FAC2FB395AF93F9D0A2EB94
:10615000B2E0CA0FDB1F50912C0152955E7E219652
:10616000AF91A395AE1711F05993FBCFFF91EF912B
:10617000DF91CF91CF93DF93EF93FF93BD2FAC2FA0
:10618000BE5FDED05EEE59935DEEA395AE1711F0C3
:106190005993FBCF5FEE5993FF91EF91DF91CF9130
:1061A000BF91AF915F9108950F931F932F933F93EA
:1061B000AF93BF93CF93DF93DE010FEFCE1B10F4AD
:1061C0000195C1951FEFDF1B10F41195D195CD17E7
:1061D00060F000C02C2F26950ADEAE1789F0A00FC4
:1061E0002D1BD0F7B10F2C0FF7CF2D2F2695FFDDEC
:1061F000BF1731F0B10F2C1BD0F7A00F2D0FF7CF29
:10620000DF91CF91BF91AF913F912F911F910F914E
:106210000895AF93A82DA73EE9F3A82DA73EE9F76F
:10622000AF910895EF93FF93AF93A0931D01FBE807
:10623000A6FDFCE8F0932F01AF73AA0FFDE8E0E89C
:10624000EA0FF21DA591A0931A01A591A0931B013D
:1062500020921C012092180120921901AF91FF9108
:10626000EF91089520921701409117014030E1F31A
:106270009DC0409116014030E1F708955FD0A2EB38
:10628000CA0FA2E0DA1FA881BA2FAF93A171BE7E18
:10629000B295BA2BAF91209217014091170140306F
:1062A00041F4409110014B3110F4A883F6CFB8832C
:1062B000F4CFA8837BD042C03F933DED52D02092D3
:1062C0001701409114014470431749F0403021F404
:1062D0000E94EA06342F03C00E941007342F409119
:1062E0001701403061F4409110014B3120F4488196
:1062F0004F774883E6CF488140684883E2CF588192
:106300005F7758833F910895D1E0C3EDCA0FD21D46
:106310002092170140911701403061F44091100123
:106320004B3120F448814F774883F4CF488140684F
:106330004883F0CF58815F7758830895AA2DBB2DED
:10634000DEE1BD9FD1E0C8ECCA0FD21DC00DD11D4A
:106350000895F6DF0F9302EBC00F02E0D01F0F91FC
:106360000895D3E2BD9FD2E0C4E3CA0FD21DC00D91
:10637000D11D0895AA2DBB2DAA95B39525CDBF9308
:10638000B0910C01B4FD0EC0BFEFB1B900001A9975
:10639000FECF42B9B4E6BA95F1F72998B4E6BA95BA
:1063A000F1F7299ABF9108954F9108954F93409125
:1063B0002D0141FFF9CF4D7F40932D01FF93EF93C6
:1063C000DF93CF9340913E01403029F44091290161
:1063D00047FF13C02FC04F9347E4D8D04F914F933E
:1063E000405DD4D04F91413009F45AC0423009F495
:1063F00070C0433009F48CC09EC044E50E94C63290
:106400004AE00E94C632C8ECD1E0FEE2EEE14881EB
:106410004295ADD04991ABD0EA95C9F74AE00E94C8
:10642000C632FA9599F7CF91DF91EF91FF914F9195
:106430004427089545E40E94C6324091400194D01B
:106440004AE00E94C632C8ECD1E0F3E0E3E24881C2
:1064500042958DD049918BD0EA95C9F74AE00E94C8
:10646000C632FA9599F7E3E2F0912E01EF9FC00D45
:10647000D11DF0E1E3E248814F77429578D0499110
:106480004F7775D0EA95B9F74AE00E94C632FA957F
:1064900089F7CF91DF91EF91FF914F9144270895B4
:1064A0004091000161D0409101015ED04AE06ED080
:1064B000C8ECD1E0F4E7E5E14881429558D0499134
:1064C00056D0EA95C9F74AE00E94C632FA9599F784
:1064D000E0CF4091000148D04091010145D040916A
:1064E000020142D0409103013FD04AE04FD0C8ECB6
:1064F000D1E0F4E5EEE14881429539D0499137D0B9
:10650000EA95C9F74AE00E94C632FA9599F7C1CFD9
:106510004AE03CD0C8ECD1E0FAE3EAE24881429597
:1065200026D0499124D0EA95C9F74AE00E94C632A4
:10653000FA9599F7AECF4091000116D04091010134
:1065400013D04AE023D0C8ECD1E0F0E4E0E1488188
:1065500042950DD049910BD0EA95C9F74AE00E94C7
:10656000C632FA9599F795CF4295469547704F7088
:10657000405D4A3308F0495F0C94C632BF93B2E0E5
:10658000A03009F0B064B4BDBF910895BF93B0913D
:106590002501B030E1F740932601BA95B09325016B
:1065A000BF910895BF93B0912701B030E1F7BA953C
:1065B000B0932701B0912701B030E1F74091280155
:1065C000BF910895BF93B0912701B030E1F7BA951C
:1065D000B0932701409116014D3E41F0B091270143
:1065E000B030C1F740912801BF9108954BE1BF91B0
:1065F0000895DF93CF93BF93AF93FF93EF93CEE0D4
:10660000D7E0E8E7F6E632D0EF91FF91FF93EF9302
:10661000CCE5D4E0B0911401B2FD7E9616F026D000
:1066200001C01ED040911601A1E04D3E69F0A2E0EC
:10663000413F51F0A3E0423F39F0A4E0433F21F055
:10664000A5E0443F09F0E0CFB0911401B2FDAB5F8B
:106650004A2FEF91FF91AF91BF91CF91DF910895B4
:10666000BEE1A191A993BA95E1F70895BEE1A59184
:10667000A993BA95E1F708954E4E4E4E4E4EC0C0C6
:10668000C0C0C0C08080808080802E2E2E2E2E2EF6
:106690006E6E6E6E6E6EACE5B0910C01B3FDAFE543
:1066A000ACBDACE5A093B800A0E0B2FDA1E0A09322
:1066B000B9000895FF93EF930F93E0911E01A0910D
:1066C0001F01B0912001F09121010027E2FD00950A
:1066D000E5FD0095A4FD0095F7FD0095001FEE1F58
:1066E000AA1FBB1FFF1FE0931E01A0931F01B093C1
:1066F0002001F09321010F91EF91FF910895FF93F5
:10670000EF93DF93CF93BF93AF934F935F936F93C9
:106710007F934F925F926F927F922F9320913E01D1
:1067200040904601509049016090480170904B01A3
:106730005091470160914A01A22FA370E52F660F87
:10674000EE0FA33031F0660FEE0FA23011F0660F9E
:10675000EE0FF62FA0914C01A13071F4E20147D069
:10676000803011F08FE133C0E30141D0803011F06F
:1067700080E22DC065D02BC0A23091F4E20137D069
:10678000803011F08FE123C0E30140D0803011F060
:1067900082E11DC0ACE3BDE06A0E7B1E75D017C060
:1067A000A33011F085E113C0A52DA33010F082E1D4
:1067B0000EC0ACE3BDE04A0E5B1EF2015191619147
:1067C000E30115D0803011F080E201C067D02F9135
:1067D0007F906F905F904F907F916F915F914F91FD
:1067E000AF91BF91CF91DF91EF91FF910895CE0FBF
:1067F00010F48FE10895A0914401CA17D0F7DF0F7C
:10680000C0F3B0914501DB17A0F70895659FC00D57
:10681000D11D2296D33008F082E10895A22F509125
:10682000470160914A01E52F660FEE0FA33031F06A
:10683000660FEE0FA23011F0660FEE0FF62F0895DF
:10684000571478F0D20134D0E0E8FBE064D0D301F3
:106850002FD0E0E8FBE08CD0539473946A9591F7C5
:106860000895560E760E5A947A94D20121D0E0E81B
:10687000FBE051D0D3011CD0E0E8FBE079D05A9482
:106880007A946A9591F70895F30151936193D20137
:106890000FD041D053946A95D1F70895F2015191E8
:1068A0006191D30105D064D073946A95D1F70895AE
:1068B0006F93C8ECD1E0213011F465E103C02530BD
:1068C00069F460E1B69FC00DD11D6A2F669566958B
:1068D0006695C60FD21D4A2F6F910895223069F434
:1068E0006EE1B69FC00DD11D6A2F66956695C60FE5
:1068F000D21D4A2F440F6F9108956AE2B69FC00DD2
:10690000D11D6A2F66956695C60FD21D4A2F440F7A
:10691000440F6F9108957F936F93BF93AF93652F4B
:10692000742F777049F4A991A1936A95E1F7AF911B
:10693000BF916F917F910895B0E8713019F0B695CD
:106940007A95FBCF7727A991AB9F703019F0A29170
:10695000A029A193119273957617A9F7A991AB9FDE
:10696000A291A029A193AF91BF916F917F910895BA
:106970007F936F93BF93AF93652F742F777049F414
:10698000A191A9936A95E1F7AF91BF916F917F9122
:1069900008950F931F930FEF11E0000F110F7A95D9
:1069A000E1F7652F7881009570230095A191A19F53
:1069B000072A0992712D6A95C9F768816023672BB0
:1069C00069930F911F91AF91BF916F917F9108953E
:1069D000BF93AF934F939927A42F0E94C12C0E947D
:1069E0003C2D4F91AF91BF910895AF93BF93EF931B
:1069F000FF935F936F930F931F932F9310E020E00B
:106A0000FAE8EE27509147015F7760914A016F776E
:106A10000491059FA12DE0950491E095069FB12D6D
:106A2000A11729F4B21719F4E39591F724C01A2F8E
:106A30002B2FA0914601B0914901A10FB20F0E94E6
:106A4000F72EA0914601B0914901A10FB21B0E94FF
:106A5000F72EA0914601B0914901A11BB21B0E94E3
:106A6000F72EA0914601B0914901A11BB20F0E94DF
:106A7000F72EE39569F62F911F910F916F915F911A
:106A8000FF91EF91DF91AF910895AF93BF93EF9393
:106A9000FF935F936F930F931F932F933F932FEF6A
:106AA000FAE8EE27509147015F7760914A016F77CE
:106AB0000491059FA12DE0950491E095069FB12DCD
:106AC000B21721F4E395A1F73F91D5CF1A2F2B2FC1
:106AD000A0914601B09149013A2FB21BA11B310F81
:106AE0000E94F72EB20FB20F0E94F72EB21BB21BFC
:106AF000A3953A17A8F7E395D9F63F91BCCFFF913C
:106B0000EF91EE0FFF1F5BD03197F695E795319629
:106B1000EF93FF93C8E7D1E040912C014F93FF938F
:106B2000EF9361D00E94CB2E0B0920505245535356
:106B300020454E5445522000EF91FF914F914093D4
:106B40002C0190DB4A3EE9F794DB0E94B9190895C5
:106B5000FF91EF91EE0FFF1F32D03197F695E79539
:106B60003196EF93FF93C8E7D1E040912C014F930A
:106B7000FF93EF9338D00E94CB2E0B082028592981
:106B80006573202F20284E296F200000EF91FF9180
:106B90004F9140932C0166DB493761F0493551F044
:106BA0004E3619F04E3409F0F6CF63DB0E94B91966
:106BB000442708955EDB0E94B91941E00895C8E7B3
:106BC000D1E0459146954F93477049934F91429537
:106BD0004770499358E145914993403011F05A95D7
:106BE000D1F729920895FF93EF9392E020922A0122
:106BF000A991B991B295B077A770AB0FAA0FA093E6
:106C00002C01DF93CF930E949319C2E0D8E0EBE10F
:106C1000FCE00E943630A3E0B9E00E94E42ECF9160
:106C2000DF9158E14991403051F0DF93CF935F936A
:106C30000E943D2D5F91CF91DF915A9599F7409138
:106C40002C01429540932C01EF91FF910895FF9301
:106C5000EF93DF93CF93BF93AF93C0914601D09151
:106C600049010A8119810E3118F4173108F41AD03C
:106C7000A0914801B0914B01C0914601D0914901CA
:106C8000B983AA83AE3138F4B73128F43DD073709C
:106C9000713009F076D0AF91BF91CF91DF91EF9134
:106CA000FF910895C0914601D09149010A8119814F
:106CB0002C813B81239F310F2596C00DD11DC00D26
:106CC000D11D412FE8ECF1E05EE1549FE00DF11D94
:106CD000E00FF21D522F699161935A95E1F74395A8
:106CE000431781F7412FEAE7F4E05EE1549FE00D9E
:106CF000F11DE00FF21D522F699161935A95E1F752
:106D00004395431781F70895C0914601D0914901F9
:106D10000A8119812C813B81239F310F2596C00D5B
:106D2000D11DC00DD11D7727412FE8ECF1E05EE1C8
:106D3000549FE00DF11DE00FF21D522F61916993F8
:106D40006F7009F071E05A95C9F74395431769F7D9
:106D5000E0914601F09149014081742B7083412FED
:106D6000EAE7F4E05EE1549FE00DF11DE00FF21D53
:106D7000522F619169935A95E1F74395431781F733
:106D80000895C0914601D09149010A8119812C8151
:106D90003B81310F2596412FE8ECF1E05EE1549FF5
:106DA000E00DF11DE00FF21D522F699161935A958C
:106DB000E1F74395431781F7412FEAE7F4E05EE1FD
:106DC000549FE00DF11DE00FF21D522F6991660FE7
:106DD00028F46E70462E6081607F642961935A9515
:106DE000A9F74395431749F70895AF93BF93CF93FE
:106DF000DF934F935F936F937F934F9270912C012A
:106E00004370E1F4A6E0B2E0C4E2D2E0422C07D045
:106E1000A8EBB4E0C6EDD4E0472E01D061C062E13A
:106E20005AE149914D935A95E1F7149624966A9543
:106E3000B9F75AE14D925A95E9F708954130C9F4EE
:106E4000ACE3B4E0CBE3D4E0422C07D0AEEEB6E046
:106E5000CDEED6E0472E01D043C063E159E14A911F
:106E60004E935A95E1F74E92149725976A95B1F78C
:106E700008954230E1F4ACE3B4E0CEE1D4E0422C3A
:106E800007D0AEEEB6E0C0EDD6E0472E01D028C068
:106E900062E15AE14A914E935A95E1F7149724978B
:106EA0006A95B9F75AE14E925A95E9F70895A6E026
:106EB000B2E0C7E0D2E0422C07D0A8EBB4E0C9EBC7
:106EC000D4E0472E01D00CC063E159E149914D93C4
:106ED0005A95E1F74D92259614966A95B1F7089563
:106EE0004F907F916F915F914F91DF91CF91BF91C3
:106EF000AF9108955E984CE54093B80044E8409304
:106F0000BC0044E94093BC00089544EA0EC050938D
:106F1000BB0044E80AC044EC08D05091BB0008957F
:106F200044E803D05091BB0008954093BC004091C9
:106F3000BC0047FFFCCF6091B900687F0895E5DF92
:106F4000683089F4572F550F5E70506AE0DF683162
:106F500051F45B2FDCDF683231F45A2FD8DF68320E
:106F600011F4882708958FE0CCCFCFDF6031D9F7B7
:106F7000572F550F5E70516ACADF6034A1F788271A
:106F80000895DDDF803049F4F0DF803031F4C8DF70
:106F9000683519F411968827B4CF8FE0B2CF5F938C
:106FA000CEDF5F91803031F4B2DF683219F4119690
:106FB0008827A7CF8FE0A5CFA8DF6830A9F4572F87
:106FC0005770550F5169A3DF603471F4A4DF603549
:106FD00059F4A52FA5DF683539F4BB27550FAA1F33
:106FE00008F4B09588278DCF8FE08BCF8827D830D5
:106FF00020F080E34F914F914FEF0895F7DFF9991B
:10700000FECFD2BDC1BDF89A40B521960895EEDFFE
:10701000F999FECFD2BDC1BDF89A40B4441611F41F
:107020002196089554E040BDF894FA9AF99A78941C
:10703000F999FECFF89A40B4441511F421960895B9
:10704000839580635A9579F70895AF93D7DF41937D
:10705000AA95E1F7AF910895AF934191D8DFAA9532
:10706000E1F7AF9108954EBD4DB547FFFDCF4EB549
:10707000089588272C9847EDF6DF4427F4DF2C9AF3
:107080004C7B4432B1F34C31A1F38827443A19F0D8
:107090004C3909F081E108958827EBDF803021F039
:1070A00040E040939C1008954C3911F448E0F9CF2A
:1070B00040E1F7CFF1DF403009F40895440F440F69
:1070C000440F440F4A950895AA0FBB1F4B2FCBDFE7
:1070D0004A2FC9DF422DC7DFB695A79508958030A6
:1070E00059F44F93C6DF803031F42C9845E5BBDF6F
:1070F000EBDF2C9ABEDF4F910895803059F44F9307
:10710000B8DF803031F42C9843E5ADDFDDDF2C9A19
:10711000B0DF4F910895803051F44F93AADF803053
:1071200029F42C9846E89FDFCFDF2C9A4F910895E1
:107130001196B0939D10A0939E101197ECCF7F9362
:10714000772710D07F9108957F9371E00BD0D42FD3
:1071500072E008D0C42F7F9108957F9373E002D02E
:107160007F9108958030B9F484DF8030A1F42C98A9
:1071700042ED79DFAA0FBB1FA3954B2F74DF4A2F77
:1071800072DF472F70DFB695A7956DDF6CDF6BDF81
:107190006ADF69DF2C9A08958030D1F46ADF80308D
:1071A000B9F42C9842ED5FDFAA0FBB1F4B2F5BDFBA
:1071B0004A2F59DF472F440F56DFB695A79553DF67
:1071C00052DF51DF50DF4FDFD42F4DDFC42F2C9A19
:1071D00008957F9370E010D07F9108957F9371E0C0
:1071E0004D2F0AD072E04C2FBDDF7F9108957F9321
:1071F00073E0B8DF7F9108958030A1F44F9339DFB9
:107200004F91803079F42C984F9347E82CDF442736
:107210002ADF41E028DF472F26DF4F914F9323DFFE
:107220002C9A4F910895803091F423DF8030D1F76C
:107230002C984F9347E817DF442715DF40E013DF12
:10724000472F11DF4F914F930EDF2C9A4F910895E6
:107250008030D1F4DF93CF934F935F930ADF803078
:1072600079F42C9847E8FFDE4427FDDE4427FBDE57
:1072700040E0F9DE55274991F6DE5A95E1F72C9A60
:107280005F914F91CF91DF9108958030B1F44F938A
:107290005F93EFDE803079F42C9847E8E4DE4427F2
:1072A000E2DE4427E0DE40E0DEDE55274FEFDBDEA6
:1072B0005A95E1F72C9A5F914F9108958030E1F44F
:1072C000DF93CF934F935F93D4DE803089F42C9873
:1072D00046EDC9DE4427C7DE4427C5DE40E0C3DEF5
:1072E0004427C1DE5527BFDE49935A95E1F72C9A12
:1072F0005F914F91CF91DF910895BF93AF93DF934B
:10730000CF934F935F937F93C7DE403041F47F91DB
:107310005F914F91CF91DF91AF91BF910895B5DF0C
:107320004FE057DF442763DFAA27BB27F4DE11961F
:107330004DEFCA2FCF70C13009F44CEF4ADF44271C
:1073400056DFCC27DD274ADFE6DE1196A03019F4A0
:1073500045EE0E943D2D40919C10B41749F7D7CFC0
:10736000BF93AF93DF93CF934F935F937F9394DE5D
:10737000403091F47F915F914F91CF91DF91AF9128
:10738000BF910895B42FAA271197E7DEC42FBB271A
:10739000AA27E3DE4C1731F4A2DEDFDE439527DFB8
:1073A000BADEE8CF1196D9DE4C17E1F7F5CFDF93BF
:1073B000CF934F9394DE4DEFCA2FCF70C13009F4B5
:1073C0004CEF07DFC1DE219609DF5FDFA4DE4F91BE
:1073D000CF91DF910895FF93DF93CF93BF93AF9346
:1073E000AA27BB27ED0158DE4030A1F0F42FA7DE1D
:1073F0004C3F41F04D3F31F04B3A21F04F3018F007
:10740000403908F421961196BF1789F74427DF17F2
:1074100009F441E0AF91BF91CF91DF91FF910895C1
:107420000F93BF93AF934F93AA27BB27ED01FD01A5
:1074300033DE403099F0042F82DE4D3F49F4DF9374
:10744000CF9382DE4D2FCF91DF914F3F21F02196D8
:107450004C3F09F431961196B01771F74F91AF91E7
:10746000BF910F910895FF93EF93DF93CF934F93C5
:107470002F9312DE4030A9F0AA27BB2760DE242F0D
:10748000B0919D10A0919E1040910801B41710F08A
:10749000A2E0BB27FD0153DE4D3F51F455DED2176C
:1074A00038F42F914F91CF91DF91EF91FF91089593
:1074B000159640919C10B41709F4BB27BF1759F7D4
:1074C000AE1749F7AA27BB270ADE39DE4F3F31F056
:1074D000405F242F7EDE1FDEDF01DDCFAFEFBFEF89
:1074E000E0CFFF93EF93DF93CF93BF93AF934F938F
:1074F0005F936F937F93D0DD403061F481E17F91A2
:107500006F915F914F91AF91BF91CF91DF91EF91CB
:10751000FF91089551D0B41710F08BE1F0CF0FDE3A
:107520004C3F11F087E1EBCF40915A01403011F40C
:107530008BE1E5CF413810F08BE1E1CF71DFD03046
:1075400021F4C41710F488E1DACFC0E8DBE050E0A2
:107550006FEF69935A95E9F798DE1196B0939D10F5
:10756000A0939E1040915A01C0E8DBE04F937BDF6F
:10757000B993A9934BEA2DDEDF93CF93E5DD2196F6
:107580002DDECF91DF91E9DD32DED2DDE9DE4F91F4
:107590004A9561F711D0C0E8DBE05ADE40915C010A
:1075A00018DEDF93CF93D0DD219618DECF91DF91E7
:1075B000D4DD1DDEB0DDA3CFA0915801A295BA2F76
:1075C000A07FBF7011960895BF93AF93DF93CF93C1
:1075D0004F935F937F937727EFDFB1DD4C3F69F0E7
:1075E000DBDDDF3F49F0BF93AF93DE01E0DEAF911B
:1075F000BF91B6DE7F5FA1F7DADE7F915F914F9199
:10760000CF91DF91AF91BF910895BF93AF93DF9377
:10761000CF934F935F937F932F93AA27BB2729DDA7
:107620008EDD242FC9DF8BDD4C3F51F489E12F9192
:107630007F915F914F91CF91DF91AF91BF9108956D
:1076400070915A01703810F08BE1F1CFA5DDDF3F6A
:1076500011F48BE1ECCFDE01CCE3DDE040915C0185
:10766000413009F4D395423009F4DE5FF1DDDF9358
:10767000CF936ADDD21759F02196B0DDCF91DF911B
:107680005EDDA7DD6ADDB3DD46DD6ADED0CF8FDEED
:10769000EADE5ADD2196A2DDCF91DF914BEA99DD3A
:1076A0005CDDA5DD38DDED0187DF19DD70915A0164
:1076B000770F4D2FB8DD73954C2FB5DD40DD89DD9B
:1076C0004CDD95DD28DDB3CFBF93AF93DF93CF9330
:1076D0004F935F937F9370DF32DD4C3F49F48EE12F
:1076E0007F915F914F91CF91DF91AF91BF910895BD
:1076F00070915A01703810F08BE1F2CF4DDDDF3F11
:1077000011F48BE1EDCFDE01EADCCCE3DDE040916A
:107710005C01413009F4D395423009F4DE5FCEDDDF
:10772000DFCF0004080D11161A1F23282C3035391D
:107730003D42464A4F53575B5F64686C7074787C77
:107740007F83878B8F92969A9DA1A4A7ABAEB1B58C
:10775000B8BBBEC1C4C6C9CCCFD1D4D6D9DBDDDF5E
:10776000E2E4E6E8E9EBEDEEF0F2F3F4F6F7F8F92F
:10777000FAFBFCFCFDFEFEFFFFFFFFFF000000CC5C
:10778000C000333000FFF000000CCCCCCCCC333C3C
:10779000CCFFFCCC000333CCC333333333FFF333A0
:1077A000000FFFCCCFFF333FFFFFFFFFA5A5A506CE
:1077B000FF6000000000000000000000000000006A
:1077C00000000000000000000000000000000000B9
:1077D0000EAE000004E000AAE800EE4E00000044F7
:1077E0004040AA000066FF666842C4A248A00000AC
:1077F000004400004888404222400A4A0004E40055
:1078000000048000E000000040224880EAAAE04C2A
:1078100044E0E2E8E0E2E2E0AAE220E8E2E0E8EACE
:10782000E0E24880EAEAE0EAE2E0040400040480DE
:107830002484200E0E00842480C268E400EEE04A16
:10784000AEA0CACAC0688860CAAAC0E8C8E0E8C8D2
:107850008068EA60AAEAA0E444E0E22A60AC8CA076
:107860008888E0AEAAA0CAAAA04AAA40EAE8804A4C
:10787000AA60EAECA068E2C0E44440AAAAE0AAAA8E
:1078800040AAAEA0AA4AA0AA4440E248E0644460EC
:1078900004A400C444C04A00000000E04400004AC0
:1078A000AEA0CACAC0688860CAAAC0E8C8E0E8C872
:1078B0008068EA60AAEAA0E444E0E22A60AC8CA016
:1078C0008888E0AEAAA0CAAAA04AAA40EAE8804AEC
:1078D000AA60EAECA068E2C0E44440AAAAE0AAAA2E
:1078E00040AAAEA0AA4AA0AA4440E248E024C4208C
:0C78F0004444448464808842208CEC8076
:1086000000F900F5F3F1F2FC00FAF8F6F4EB5E0085
:10861000F7000000007131000000797361773200CB
:108620000063786465343300002076667472350028
:10863000006E6268677A360000006D6A7537380030
:10864000002C6B696F303900002E2D6C00707E009D
:1086500000000000002700000000EA2B00230000BB
:10866000003C00000000EC00003100343700000046
:10867000302C32353638ED00FB2B332D2A390000F3
:1086800000F900F5F3F1F2FC00FAF8F6F4EB000063
:10869000F70000000051210000005953415722000B
:1086A00000435844452440000020564654522500BB
:1086B000004E4248475A260000004D4A552F2800D8
:1086C000003B4B494F3D2900003A5F4C00503F00B2
:1086D00000000000006000000000EA2A00270000FF
:1086E000003E00000000EC000031003437000000C4
:1086F00030E932353638ED00FB2B332D2A390000B6
:108700000000000000000000000000000000000069
:108710000000000000000000000000000000000059
:108720000000000000000000000000000000000049
:1087300000000000000000C000000000000000C1B8
:10874000000000000000000000002F0000000000FA
:1087500000000000000000000000EA000000C2006D
:10876000000000000000000000E100E2E000000066
:10877000E8E9E500E3E4ED00FB2BE72D2AE6000045
:1087800000000000000000000000000000000000E9
:108790000000000000400000000000000000000099
:1087A00000000000000000000000000000000000C9
:1087B000000000000000000000000000007B5B00E3
:1087C00000000000007D5D000000000000007E0051
:1087D00000000000000000000000005C000000003D
:1087E000007C00000000000000E100E2E00000006A
:1087F000EFEEE500E3E4ED00FB2BE72D2AE60000B9
:1088000000F900F5F3F1F2FC00FAF8F6F4EB5E0083
:10881000F70000000071310000007A7361773200C8
:108820000063786465343300002076667472350026
:10883000006E62686779360000006D6A753738002F
:10884000002C6B696F303900002E2F6C3B702D00AF
:10885000000027005B3D00000000EA5D007E000094
:10886000000000000000EC00003100343700000080
:10887000302C32353638ED00FB2B332D2A390000F1
:1088800000F900F5F3F1F2FC00FAF8F6F4EB000061
:10889000F70000000051210000005A5341574000EA
:1088A00000435844452423000020564654522500D6
:1088B000004E424847595E0000004D4A55262A00A6
:1088C000003C4B494F292800003E3F4C3A505F0086
:1088D000000022007B2B00000000EA7D007C0000ED
:1088E000000000000000EC00003100343700000000
:1088F00030E932353638ED00FB2B332D2A390000B4
:108900000000000000000000000000000000000067
:108910000000000000000000000000000000000057
:108920000000000000000000000000000000000047
:1089300000000000000000C000000000000000C1B6
:10894000000000000000000000002F0000000000F8
:1089500000000000000000000000EA000000C2006B
:10896000000000000000000000E100E2E000000064
:10897000E8E9E500E3E4ED00FB2BE72D2AE6000043
:1089800000000000000000000000000000000000E7
:1089900000000000000000000000000000000000D7
:1089A00000000000000000000000000000000000C7
:1089B00000000000000000000000000000000000B7
:1089C00000000000000000000000000000000000A7
:1089D0000000000000000000000000000000000097
:1089E000000000000000000000E100E2E0000000E4
:1089F000E8E9E500E3E4ED00FB2BE72D2AE60000C3
:108A0000FFFFFFFFFFFFFFFFFFFFFFFEFEFEFEFE7B
:108A1000FEFEFDFDFDFDFDFCFCFCFCFBFBFBFBFA93
:108A2000FAFAF9F9F9F8F8F8F7F7F6F6F6F5F5F4D1
:108A3000F4F3F3F2F2F2F1F0F0EFEFEEEEEDEDEC35
:108A4000EBEBEAEAE9E8E8E7E6E6E5E4E4E3E2E1BD
:108A5000E1E0DFDEDEDDDCDBDADAD9D8D7D6D5D46B
:108A6000D4D3D2D1D0CFCECDCCCBCAC9C9C8C7C63A
:108A7000C5C4C3C2C1BFBEBDBCBBBAB9B8B7B6B529
:108A8000B4B2B1B0AFAEADACAAA9A8A7A6A5A3A237
:108A9000A1A09E9D9C9B99989796949392918F8E5E
:108AA0008D8B8A898786858382817F7E7D7B7A789C
:108AB0007776747371706F6D6C6A696766656362EF
:108AC000605F5D5C5A595756545351504E4D4B4A56
:108AD0004847454442413F3E3C3B393836353332C6
:108AE000302E2D2B2A2827252422201F1D1C1A1941
:108AF00017161412110F0E0C0B09070604030100C0
:108B00000C11161A1E2225282B2D2F313233333407
:108B100034343434343434343535363738393B3CF6
:108B20003E40434547494B4D4F5152535454545482
:108B3000545351504E4C4A4745423F3D3A383634E3
:108B40003231302F2E2E2E2F303132333536383A07
:108B50003C3E4042444647494A4B4D4E4E4F505092
:108B60005050505050504F4E4D4C4B494846434149
:108B70003E3B37332F2B27221D18130D0802FDF81B
:108B8000F3EEE9E5E1DDDAD7D4D2D0CECDCCCCCB53
:108B9000CBCBCBCBCBCBCBCBCACAC9C8C7C6C4C344
:108BA000C1BFBCBAB8B6B4B2B0AEADACABABABAB98
:108BB000ABACAEAFB1B3B5B8BABDC0C2C5C7C9CB17
:108BC000CDCECFD0D1D1D1D0CFCECDCCCAC9C7C5D3
:108BD000C3C1BFBDBBB9B8B6B5B4B2B1B1B0AFAF28
:108BE000AFAFAFAFAFAFB0B1B2B3B4B6B7B9BCBE51
:108BF000C1C4C8CCD0D4D8DDE2E7ECF2F7FD02075F
:108C0000000A141D272F383F464B505457595959C5
:108C1000585654504C48433E39332E2925201C19B0
:108C200016141211111112131517191C1F222527C2
:108C30002A2C2E303132323232312F2D2B28252260
:108C40001F1C191613110F0D0C0B0A0A0A0B0C0E20
:108C500010121416181A1C1E1F2020201F1E1C196B
:108C600016120D0803FDF7F0EAE3DDD6D1CBC6C23C
:108C7000BFBDBBBABBBCBEC2C6CBD1D7DFE6EFF728
:108C80000008101920282E34393D41434445444200
:108C9000403D39342E29221C150F0802FCF7F2ED55
:108CA000E9E6E3E1E0DFDFDFE0E1E3E5E7E9EBED83
:108CB000EFF1F3F4F5F5F5F4F3F2F0EEECE9E6E3B9
:108CC000E0DDDAD7D4D2D0CECDCDCDCDCECFD1D37D
:108CD000D5D8DADDE0E3E6E8EAECEDEEEEEEEDEB3A
:108CE000E9E6E3DFDAD6D1CCC6C1BCB7B3AFABA9F6
:108CF000A7A6A6A6A8ABAFB4B9C0C7D0D8E2EBF57B
:108D000080675342352B221C16120E0C09070605EC
:108D1000040000000000000000000000000000004F
:108D20000000000000000000000000000000000043
:108D30000000000000000000000000000000000033
:108D40000000000000000000000000000000000023
:108D50000000000000000000000000000000000013
:108D60000000000000000000000000000000000003
:108D700000000000000000000000000000000000F3
:108D8000890091009A00A300AD00B700C200CE0098
:108D9000DA00E700F4000301120123013401460167
:108DA0005A016E0184019B01B301CD01E901060264
:108DB0002502450268028C02B302DC020803360376
:108DC00067039B03D2030C0449048B04D0041905E8
:108DD0006705B90510066C06CE063507A307170808
:108DE000930815099F09320ACD0A720B200CD80C82
:108DF0009C0D6B0E460F2F1025112A123F13641481
:108E0000F894A0E02A2EA1E03A2EA0E1AEBFAFEF89
:108E1000ADBFB0E0A0E0AA95F1F7BA95D9F7AAEBFB
:108E2000A4B9AFEFA5B9A0E8A7B9A0E0A8B9A0EF91
:108E3000AAB9AFEFABB9A6B1AF71A09329014B9915
:108E40005DC0B2ECB0938000B9E1B0938100F4E072
:108E5000A2FFF4E0F0938700FEEFA2FFF6EFF0939D
:108E6000860020928900FAE5F0938800A2E0A093A2
:108E70006F00A0E4A4BDA1E0A5BDA1E3A7BD209221
:108E8000C000A0E1A093C100A6E6A093C200E0EA62
:108E9000FFE87ED0A2E2B591B993AA95E1F705B7B4
:108EA000036005BF0E7F05BF7894A8EC68D0B09131
:108EB000C600B83719F0AA95C9F720C0E0ECFFE862
:108EC00067D045E140D0C8ECD1E020D046E03BD0AF
:108ED000E0E0F0E0CCE3DFE019D046E034D0CCEBCA
:108EE000DFE014D0FE3820F40E946B79329678943B
:108EF00046E029D0AEEDB1E01BD0ECCFF89405B739
:108F0000016005BF0C7F05BF0C94000028D04430E1
:108F100039F446E018D0B0912501B030E1F7EECF3A
:108F200050E81DD01CD01BD049935A95E1F717C0CB
:108F30004F2F429501D04F2F4F70405D4A3308F0BC
:108F4000495F4D930895BF93B0912501B030E1F78B
:108F500040932601BA95B0932501BF910895BF9320
:108F6000B0912701B030E1F7BA95B0932701B091E5
:108F70002701B030E1F740912801BF910895AF93E8
:108F8000A82DA73EE9F3A82DA73EE9F7AF910895D4
:108F9000C8ECD1E0A2E2B591B993AA95E1F70895A2
:108FA0004156522D436869704261736963322028CB
:108FB0004631313D557064617465205379732920C1
:108FC000426F6F746C6F61646572204572726F726C
:108FD000202845534320746F206578697429202028
:0C900000202020202020202020202020E4
:0C9C0000202020202020202020202020D8
:0CA80000202020202020202020202020CC
:0CB40000202020202020202020202020C0
:0CC00000202020202020202020202020B4
:0CCC0000202020202020202020202020A8
:0CD800002020202020202020202020209C
:0CE4000020202020202020202020202090
:10F000000C94004700000000000000000000000019
:10F0100000000000000000000000000000000000F0
:10F0200000000000000000000000000000000000E0
:10F03000000000000C941C784F935F936F93FF9334
:10F04000EF93DF93CF93BF93AF930F921F92FFB7CE
:10F05000FF93C8E0D1E0B9A5B7FF5C98B7FD5C9A13
:10F060004B99BE7F4B9BB160B9A7830C921CE9A161
:10F07000F92DF03029F4F82DFA3010F1F63EF8F0C1
:10F08000FCE0E2FFFDEE8F1639F45E98E3FF17C057
:10F09000B2E8B093800013C0F1E1E2FFF3EF8F1606
:10F0A00039F45E9AE3FF0BC0B2ECB093800007C066
:10F0B000F9E3E2FFF7E08F1611F4882499242CC0BD
:10F0C000A0918400AA3FE0F3AB3F00F0AC3F00F01A
:10F0D000AD3F00F0AE3F00F0A8ECB1E0F6EFF80D68
:10F0E000C0E2ED91549140E060E848B9ED9156FDE1
:10F0F00066B90000000055FD66B9049054FD66B97C
:10F10000CA95000053FD66B90000000052FD66B9C3
:10F11000502D59F7000028B814D0E091C600E6370A
:10F1200011F40C947E47FF91FFBF1F900F90AF9199
:10F13000BF91CF91DF91EF91FF916F915F914F91CF
:10F140001895A0913101E0912701E03091F0EF3F57
:10F1500021F4A0FD0EC0EEE30CC0EA95F5EFB491EA
:10F16000B5FF07C0B0912801B695A0FBB7F9B093E1
:10F170002801E0932701E0912501E03091F0EF3F75
:10F1800019F4E8E4AF770DC0EA95F5EFB491B4FF58
:10F1900008C0B0912601B0FB0894B795A7F9B093C9
:10F1A0002601E0932501A09331010895A09131013A
:10F1B000E0912701E03091F0EF3F21F4A0FD0EC077
:10F1C000ECE70CC0EA95F5EFB491B7FF07C0B0913A
:10F1D0002801B695A0FBB7F9B0932801E093270169
:10F1E000E0912501E030E9F2EF3F19F4E0E9AF7773
:10F1F000D8CFEA95F5EFB491B6FFD3CFB091260101
:10F20000B0FB0894B795A7F9B0932601CACF4091F7
:10F210000C01C8EFD7E00E9407380895C8EFD7E087
:10F220000E94FE3740930C010895FF93EF93DF9304
:10F23000CF93AF93F2D0E0933401F0933501AF91C7
:10F24000CF91DF91EF91FF910895E0E0F0E9C0E008
:10F25000DCE0A42FA03021F0EC0FFD1FAA95FACF1F
:10F260000895E0913401F0913501A0E2A99FE00DED
:10F27000F11DB096C0EAD1E0A0E2B591B993AA958C
:10F28000E1F7BFEFB993089547B740FDFDCFB7BF92
:10F29000E89547B740FDFDCF089547B746FF08956D
:10F2A000B1E1F2DFFACFF8944E2F407E19F4B3E0CB
:10F2B000EBDFF3DFA0E109901990B1E0E5DF3296D2
:10F2C000AA95C9F7E03009F008953297B5E0DCDF80
:10F2D000E4DF32960895F8944F93BF93AF93B3E071
:10F2E000D3DFDBDF3297CCE3DFE0A0E83296099092
:10F2F0001990B1E0C9DFAA95C9F7B5E0C5DFCDDF48
:10F30000AF91BF914F910895E0913401F091350193
:10F31000B097ACE0B591B993AA95E1F7A091290116
:10F32000A7FD0895A6EAB2E0CA0FDB1FACE0B091DA
:10F330002C01B993AA95E9F70895E0E0F0E9A0E07F
:10F34000BCE0492F403029F3EA0FFB1F4A95FACF62
:10F35000F89461D0C0EAD1E0A3EDB1E05CE04D915A
:10F3600049935A95E1F754E140E2B9935A95E9F788
:10F37000A09799DF9927B3E2B99FA4E3B2E0A00D6B
:10F38000B11DC8E7D1E050E24D9149935A95E1F79C
:10F39000299250E24A91403219F428825A95D1F7C5
:10F3A0000E94FB17C0EAD1E07EDF93959F3519F7E5
:10F3B0007894089530D0A3EDB1E05CE045914D9391
:10F3C0005A95E1F77496992750E2A0EAB1E0459189
:10F3D0004D935A95E1F7A8E7B1E040E253E24D932F
:10F3E0005A95E9F7FF93EF939F930E94E5189F9139
:10F3F000EF91FF91C8E7D1E0B3E2B99FA1E3B2E09A
:10F40000A00DB11D53E249914D935A95E1F79395A3
:10F410009F35D1F6089540913D01E0E0F0E9477055
:10F420004295A0ECA49FE00DF11D0895CCE3DFE030
:10F4300040E250E259934A95E9F740EF5FEF599364
:10F440004A95E9F7E8DF47DF3296CCE3DFE040E2B8
:10F450005FEF59934A95E9F74BE04F933CDF3296C3
:10F460004F914A95D1F778940895472F4770D5DF8B
:10F47000FF93EF93D0DFAF91BF914CE04F93CCE37C
:10F48000DFE040E0559159934A95E1F7FF93EF9300
:10F49000FD0121DF3296DF01EF91FF914F914A95F7
:06F4A00069F7789408955D
:10F50000010101010101210101010101013181011B
:10F510000100003100010101010131C101010101BE
:10F520003101010101010131C1010101013101017B
:10F530000101010131C101010101110101010101BB
:10F540000111C1010101010101010101010101C11B
:10F55000010101010101010101000101C1010101DC
:10F56000010101010101010001C1010101010100CD
:10F57000010101010101410001010101010101003D
:10F58000000000400000000000000000000000003B
:10F59000000000000000000000000000000000006B
:10F5A000000000000000000000000000000000005B
:10F5B000000000000000000000000000000000004B
:10F5C000000000000000000000000000000000003B
:10F5D000000000000000000000000000000000002B
:10F5E000100000000000000000000000000000000B
:10F5F00020000000000000000000000000000000EB
:10F60000009010800090108000901080009010807A
:10F61000FC28288004C0145028282800000000007E
:10F6200000000000000000000000000000000000DA
:10F6300000000000000000000000000000000000CA
:10F6400000000000000000000000000000000000BA
:10F6500000000000000000000000000000000000AA
:10F66000000000000000000000000000000000009A
:10F67000000000000000000000000000000000008A
:10F6800028C004C0000C60000000000000000080E2
:10F69000C0A0888400000000000000002088FCB4A6
:10F6A0000028000008A08080000004C028800024FA
:10F6B00000008000000044288000C004C41800003E
:10F6C000000000000000000000000000000000003A
:10F6D0008090808008A084408080C8A400004C8472
:10F6E0000000000000008000C004FC1C00802828EE
:10F6F000280000002828002828282800002CE8904E
:10F700000090108000901080009010800090108079
:10F710007C444480A8A814504844440024000000BD
:10F7200000183C3C185028280C3000000000000055
:10F73000241824400C401440242400000C003024E1
:10F7400024244424444040246424106460646424D9
:10F7500044244424406464646464404800481800BD
:10F76000300060000400140060180C6028000000E5
:10F7700000000000300000000000000C18306000A5
:10F7800028A004C06C109000000000000000008061
:10F79000C0A08884000000000000008040847C58E5
:10F7A000182800001090808004C004C028FC287C29
:10F7B00000440C00000044EC8000C004C42400009D
:10F7C0000000000000000000000000000000000039
:10F7D0008088A41010908440C004C8A400008C80CD
:10F7E000287C00808000C090E44CFC4C0000244841
:10F7F000280000002828002828282800002CE8C01D
:10F800000090108000901080009010800090108078
:10F81000FC44448080801450444444283C00000050
:10F8200000183C3C20546C181818181800000004EC
:10F830006428640C14603064646428281800186418
:10F84000646464646460606464180C6C605864642C
:10F8500064646464186464646464046000183C0054
:10F860001800600004003400600000601800000010
:10F870000000000030000000000000181818601898
:10F88000449008A08010900000000000000000805C
:10F89000C0A0888400000000000080804084FCB488
:10F8A0002428282820888080A4A00C60448044401C
:10F8B00000440C40844444800000C0046C24004494
:10F8C0000000000000000000000000000000000038
:10F8D0008084BCB020888820D834C8A440848C8020
:10F8E0002C7C00C4C444C018FC1CFC1C0080208874
:10F8F000280000002828002828282800002CE8A03C
:10F900000090108000901080009010800090108077
:10F910007C808080808010908480804424186424BF
:10F9200000183C40780C7830300C7C180000000C3B
:10F93000681804183C44600C6464282830400C04A7
:10F94000046464606460606064180C78607C546473
:10F9500064646460186464643C640C60301864001F
:10F960000C2444242C2430207428146C185C742437
:10F970004824742448646464646440181818300C83
:10F9800044881090800C600000000000000000809F
:10F99000C0A08884000000000080808080807CEC13
:10F9A000404444442088408490A00C6044FC286477
:10F9B00000440C40844444280000C0046C240080AF
:10F9C0000000000000000000000000000000000037
:10F9D0008080BC1040848820E82CC8A480804C849F
:10F9E000EC2400C4EC44E40CFC4CE44C0080208883
:10F9F000280000002828002828282800002CE8E4F7
:10FA00000090108000901080009010800090108076
:10FA1000FC808080B098109080ECEC44003C6464E2
:10FA20000018003C24183000300C2440004000181E
:10FA30007C180C0C6C044418242000006000040C9A
:10FA40002C6444606444447040180C50607C7C64B6
:10FA50004464442418646464183C18607C180000F2
:10FA6000000464606864486454180C78187C54641A
:10FA70006C6C5460306464643C640C30180C188006
:10FA8000808410906C0C600000000000000000807A
:10FA9000C0A0888400000000808080808080FCB44A
:10FAA0001880442840844084808418308080282432
:10FAB00000440C40844444440000C00428241880BE
:10FAC0000000000000000000000000000000000036
:10FAD000A4B0BC4080808080E82CC8A488104084FA
:10FAE000E42400C4EC44FC34FC64C004808020881E
:10FAF000288020882088808020888020882CE8F03A
:10FB00000000000090909090101010108080808075
:10FB10007C8080801090B098408080440040646475
:10FB2000001800401C307800300C7C182800003091
:10FB300054181804400464186404282830400C1831
:10FB40007C4064606460606464180C78606468641D
:10FB5000607C780418643C7C3C1830600C18000011
:10FB6000002064606440306464180C50187C646445
:10FB70006C6C602430646464182C181818180C0C11
:10FB8000808420886C0C6000000000000000008071
:10FB9000C0A08884000000008080808080807CEC91
:10FBA00018008044408440848080301880FC801895
:10FBB00000448040844444440000C004280024449D
:10FBC0000000000000000000000000000000000035
:10FBD000BCD0A41084404084E82CC8A44C8480800D
:10FBE000482400C4EC44FC34E44CC00480802088E9
:10FBF000288020882088808020888020882CE82801
:10FC00000000000090909090101010108080808074
:10FC1000FC8080801090808084C4A8440000643CF4
:10FC20000000003C44686C00181818181800286080
:10FC3000641830640C646430640C281818001800D0
:10FC40007C6464646460606464186C6C60646464A4
:10FC500060686C6418643C7C641860600018000084
:10FC6000006464646460302064180C781864646410
:10FC7000482460043C683C7C3C0830181818041880
:10FC80004488208880109000000000000000008060
:10FC9000C0A0888400000080808080808080FCB4C8
:10FCA000400080804084208880843018DC80284098
:10FCB00000446040844444280000C0046C0024C414
:10FCC0000000000000000000000000000000000034
:10FCD000BCB0808084402088E44CC4C44C848080C4
:10FCE000282400C4EC44FC34C004C004800028284C
:10FCF000280028280000280028282820882CE83000
:10FD00000000000090909090101010108080808073
:10FD10007C4480441450808044EC442800004458C3
:10FD20000018003C18082C000C300000300028009F
:10FD3000242440240C242430242800300C003018C3
:10FD4000246444244440602464242864406464247B
:10FD5000602C64241824182464184048004800408B
:10FD6000002044242424300464246C6C246464241F
:10FD7000600C6044182C183C6404400C18300400DB
:10FD8000449040848010900000000000000000803B
:10FD9000C0A08884000080808080808040847C585F
:10FDA000240080288080208890A0600CDCFC44180F
:10FDB00000446040844444EC0000C0046C00240013
:10FDC0000000000000000000000000000000000033
:10FDD000BCB0808080801090D094C0048C8040841F
:10FDE000284000C4C444E434C00480808000282833
:10FDF000280028280000280028282820882CE830FF
:10FE00000000000090909090101010108080808072
:10FE1000FC4480441450A8A84080440000006000C6
:10FE200000000000000000000000000000000000D2
:10FE300000000000000000000000000000000000C2
:10FE400000000000000000000000000000000000B2
:10FE500000000000000000000000000000000000A2
:10FE60000000000000000024000028000000000046
:10FE700060080000000000000024000000000000F6
:10FE800028A080806C0C6000000000000000008052
:10FE9000C0A0888400808080808080804084FCECCA
:10FEA0001800444480801090A4A0C004DC806C3C06
:10FEB00000446000004400800080C004C4002400AE
:10FEC0000000000000000000000000000000000032
:10FED000A4B08080844008A0C8A480808C800000EA
:10FEE000444000808000C034C00400000000282886
:10FEF000280028280000280028282824482CE8006A
:10FF00000000000090909090101010108080808071
:10FF10007C2880281450109080EC28000000C0003D
:10FF200000000000000000000000000000000000D1
:10FF300000000000000000000000000000000000C1
:10FF400000000000000000000000000000000000B1
:10FF500000000000000000000000000000000000A1
:10FF60000000000000000000000000000000000091
:10FF70000000000000000000000000000000000081
:10FF800028C08080000C600000000000000000809D
:10FF9000C0A08884808080808080808020887C5879
:10FFA00000004480808008A004C0C0048CFCA858D5
:10FFB00000006000004400280080C004C40000006D
:10FFC0000000000000000000000000000000000031
:10FFD0008080000084400000C8A400004824000085
:10FFE000000000000000C004E44C0000800028284D
:10FFF000280028280000280028282828282CE80085
:00000001FF
